:020000040000FA
:040800002AEF08F0E3
:1008100003B213EF05F0F2B431EF05F09EB039EFFB
:1008200005F09EB241EF05F0F2A81AEF04F0F2B223
:1008300025EF04F0F2A620EF04F0F2B022EF04F06E
:10084000D9EF07F0F296F290FF00CD90F2929EA0C1
:100850002FEF04F00101533F2FEF04F0542BAEC1F2
:10086000B2F1AFC1B3F1B0C1B4F1B1C1B5F1AAC138
:10087000AEF1ABC1AFF1ACC1B0F1ADC1B1F1A6C148
:10088000AAF1A7C1ABF1A8C1ACF1A9C1ADF1A2C158
:10089000A6F1A3C1A7F1A4C1A8F1A5C1A9F19EC168
:1008A000A2F19FC1A3F1A0C1A4F1A1C1A5F19AC178
:1008B0009EF19BC19FF19CC1A0F19DC1A1F196C188
:1008C0009AF197C19BF198C19CF199C19DF1CECF4E
:1008D00096F1CFCF97F153C198F154C199F1CF6AF6
:1008E000CE6A0101536B546B9E90CD800FBC0F8E6E
:1008F0000FBA7EEF04F00F8AD9EF07F00F8C0FBE0E
:10090000BAEF04F096C19AF197C19BF198C19CF19E
:1009100099C19DF19AC19EF19BC19FF19CC1A0F12B
:100920009DC1A1F19EC1A2F19FC1A3F1A0C1A4F1FB
:10093000A1C1A5F1A2C1A6F1A3C1A7F1A4C1A8F1CB
:10094000A5C1A9F1A6C1AAF1A7C1ABF1A8C1ACF19B
:10095000A9C1ADF1AAC1AEF1ABC1AFF1ACC1B0F16B
:10096000ADC1B1F1AEC1B2F1AFC1B3F1B0C1B4F13B
:10097000B1C1B5F101015E6B5F6B606B616B96514C
:100980005E2797515F2398516023995161239A51B3
:100990005E279B515F239C5160239D5161239E5193
:1009A0005E279F515F23A0516023A1516123A25173
:1009B0005E27A3515F23A4516023A5516123A65153
:1009C0005E27A7515F23A8516023A9516123AA5133
:1009D0005E27AB515F23AC516023AD516123AE5113
:1009E0005E27AF515F23B0516023B1516123B251F3
:1009F0005E27B3515F23B4516023B5516123D89072
:100A00000101613360335F335E33D890010161339C
:100A100060335F335E33D8900101613360335F33FD
:100A20005E33D9EF07F00392ABB2AB98AB8803010A
:100A300003EE00F080517F0BE92604C0EFFF802B0E
:100A40008151805D700BD8A48B8200008051815D44
:100A5000700BD8A48B9281518019D8B40790D9EF2C
:100A600007F0F2940101453FD9EF07F0462BD9EF8B
:100A700007F09E900101533FD9EF07F0542BD9EFB7
:100A800007F09E92040062A146EF05F007B498EFCC
:100A900005F007B098EF05F01EC620F61FC621F638
:100AA0001CC61EF61DC61FF61AC61CF61BC61DF672
:100AB00006C608F607C609F604C606F605C607F612
:100AC00002C604F603C605F626C628F627C629F68A
:100AD00024C626F625C627F622C624F623C625F602
:100AE0000EC610F60FC611F60CC60EF60DC60FF6A2
:100AF0000AC60CF60BC60DF62EC630F62FC631F61A
:100B00002CC62EF62DC62FF62AC62CF62BC62DF691
:100B100016C618F617C619F614C616F615C617F631
:100B200012C614F613C615F6EEEC2BF086EC2BF07D
:100B3000077C07ACB3EF05F0C274C2B4ADEF05F0AB
:100B4000C3CFB3F5C4CFB4F50501D890B433B333F4
:100B5000D890B433B333B4EF05F0C3CF55F1C4CF5D
:100B600056F1B4EF05F0C28207B421EF06F047C199
:100B70004BF148C14CF149C14DF14AC14EF15EC142
:100B800062F15FC163F160C164F161C165F196C159
:100B9000B6F197C1B7F198C1B8F199C1B9F19AC14D
:100BA000BAF19BC1BBF19CC1BCF19DC1BDF19EC11D
:100BB000BEF19FC1BFF1A0C1C0F1A1C1C1F1A2C1ED
:100BC000C2F1A3C1C3F1A4C1C4F1A5C1C5F1A6C1BD
:100BD000C6F1A7C1C7F1A8C1C8F1A9C1C9F1AAC18D
:100BE000CAF1ABC1CBF1ACC1CCF1ADC1CDF1AEC15D
:100BF000CEF1AFC1CFF1B0C1D0F1B1C1D1F1B2C12D
:100C0000D2F1B3C1D3F1B4C1D4F1B5C1D5F1B3C5FB
:100C1000B5F5B4C5B6F5B5C5B7F5B6C5B8F50101B6
:100C200055515B2756515C23E86A5D230E2E21EF58
:100C300006F05CC157F15DC158F15B6B5C6B5D6B9D
:100C4000078E0201002FD9EF07F03C0E006F05015F
:100C50002F51000AD8B4D8EF06F005012F51010A30
:100C6000D8B462EF06F005012F51020AD8B4A3EF01
:100C700006F005012F51030AD8B4A3EF06F00501D1
:100C80002F51040AD8B4A3EF06F005012F51050A2D
:100C9000D8B4A3EF06F005012F51060AD8B4A3EF8C
:100CA00006F005012F51070AD8B4A3EF06F005019D
:100CB0002F51320AD8B460EF06F02F6BD8EF06F050
:100CC000D8EF06F0050153676DEF06F054676DEF3E
:100CD00006F055676DEF06F0566771EF06F0D8EF36
:100CE00006F057C500F158C501F159C502F15AC5C2
:100CF00003F10101010E046F000E056F000E066F77
:100D0000000E076FF7EC29F000C157F501C158F547
:100D100002C159F503C15AF5006796EF06F0016765
:100D200096EF06F0026796EF06F00367D8EF06F03D
:100D300053C557F554C558F555C559F556C55AF517
:100D40000F88D8EF06F005013067A9EF06F0D8EF5D
:100D500006F00FBEBEEF06F010A0C3EF06F00101D3
:100D60004767BAEF06F04867BAEF06F04967BAEF8F
:100D700006F04A67BEEF06F0C3EF06F007AEC3EF1A
:100D800006F0D5EF06F00501312FD8EF06F03C0E46
:100D9000316F302FD8EF06F00101000E626FE00EC8
:100DA000636FA50E646F010E656F0501306B0F88D0
:100DB0000501626B33B7DEEF06F062810CC100F112
:100DC0000DC101F10EC102F10FC103F110C104F117
:100DD00011C105F112C106F113C107F114C108F1E7
:100DE00015C109F116C10AF117C10BF135C134F172
:100DF00000C10CF101C10DF102C10EF103C10FF1EF
:100E000004C110F105C111F106C112F107C113F1BE
:100E100008C114F109C115F10AC116F10BC117F18E
:100E200034C135F101018A671DEF07F08B671DEFB3
:100E300007F08C671DEF07F08D6721EF07F051EF8A
:100E400007F08EC100F18FC101F190C102F191C193
:100E500003F10101010E046F000E056F000E066F15
:100E6000000E076FF7EC29F000C18EF101C18FF180
:100E700002C190F103C191F1006746EF07F00167ED
:100E800046EF07F0026746EF07F0036751EF07F000
:100E90008AC18EF18BC18FF18CC190F18DC191F11E
:100EA0000F80D57ED5BE69D0D6CF47F1D7CF48F1D8
:100EB00045C149F1E86AE8CF4AF1109047C100F115
:100EC00048C101F149C102F14AC103F101010A0E11
:100ED000046F000E056F000E066F000E076FF7EC33
:100EE00029F003AF1080010154A783EF07F00F9A98
:100EF0000F9C0F9E0101000E5E6F600E5F6F3D0E36
:100F0000606F080E616F010147BF93EF07F04867FC
:100F100093EF07F0496793EF07F04A6793EF07F005
:100F2000F288B8EF07F0F2985E6B5F6B606B616BF5
:100F3000966B976B986B996B9A6B9B6B9C6B9D6B8D
:100F40009E6B9F6BA06BA16BA26BA36BA46BA56B3D
:100F5000A66BA76BA86BA96BAA6BAB6BAC6BAD6BED
:100F6000AE6BAF6BB06BB16BB26BB36BB46BB56B9D
:100F7000D76AD66A0101456B466B0CC100F10DC101
:100F800001F10EC102F10FC103F110C104F111C151
:100F900005F112C106F113C107F114C108F115C121
:100FA00009F116C10AF117C10BF135C134F1D9EFBE
:100FB00007F002C0E0FF005001C0D8FF1000A6B249
:100FC000DFEF07F00CC0A9FF0BC0A8FFA69EA69CF0
:100FD000A684F29E550EA76EAA0EA76EA682F28E6A
:100FE000A694A6B2F1EF07F00C2A1200A96EA69EF5
:100FF000A69CA680A8500C2A120004012C0E826F19
:1010000024EC0BF0F2EC2AF00C50F6EC07F0E8CFF1
:1010100000F10C50F6EC07F0E8CF01F101AF16EF4C
:1010200008F00101FF0E026FFF0E036F95EC2AF02E
:10103000296722EF08F00401200E826F24EC0BF0E8
:1010400027EF08F004012D0E826F24EC0BF0BFECAB
:1010500028F01200076A0F6A106A0F010D0EC16EA8
:10106000860EC06E030EC26E0F01680E896E130EDF
:10107000926E080E8A6E8A6AF30E936E8B6A900ED9
:10108000946EF18EF19E0E6A01015B6B5C6B5D6B81
:10109000576B586BF29A0101476B486B496B4A6B6F
:1010A0004B6B4C6B4D6B4E6B4F6B506B516B526B74
:1010B000456B466BD76AD66A0F01280ED56EF28A49
:1010C0009D90B00ECD6E01015E6B5F6B606B616BCE
:1010D000626B636B646B656B666B676B686B696B8C
:1010E000536B546BCF6ACE6A0F9A0F9C0F9E9D80F4
:1010F000760ECA6E9D8202013C0E006FCC6A160EFF
:10110000F6EC07F0E8CF00F1170EF6EC07F0E8CFA9
:1011100001F1180EF6EC07F0E8CF02F1190EF6EC2B
:1011200007F0E8CF03F1010103AFB1EF08F0F2ECF3
:101130002AF0160E0C6E00C10BF0DFEC07F0170E54
:101140000C6E01C10BF0DFEC07F0180E0C6E02C143
:101150000BF0DFEC07F0190E0C6E03C10BF0DFECA7
:1011600007F000C18AF101C18BF102C18CF103C10A
:101170008DF100C18EF101C18FF102C190F103C167
:1011800091F11A0EF6EC07F0E8CF00F11B0EF6EC29
:1011900007F0E8CF01F11C0EF6EC07F0E8CF02F102
:1011A0001D0EF6EC07F0E8CF03F1010103AF07EFE6
:1011B00009F0F2EC2AF01A0E0C6E00C10BF0DFEC15
:1011C00007F01B0E0C6E01C10BF0DFEC07F01C0EDC
:1011D0000C6E02C10BF0DFEC07F01D0E0C6E03C1AC
:1011E0000BF0DFEC07F01A0EF6EC07F0E8CF00F199
:1011F0001B0EF6EC07F0E8CF01F11C0EF6EC07F041
:10120000E8CF02F11D0EF6EC07F0E8CF03F100C1C4
:1012100092F101C193F102C194F103C195F1240E41
:10122000AC6E900EAB6E240EAC6E080EB86E000E57
:10123000B06E1F0EAF6E0401806B816B0F01900EBC
:10124000AB6E0F019D8A0301806B816BC26B8B9229
:1012500081EC31F081EC31F0880EF6EC07F0E8CF4C
:1012600000F1890EF6EC07F0E8CF01F1010101AFC2
:1012700052EF09F0F2EC2AF0880E0C6E00C10BF070
:10128000DFEC07F0890E0C6E01C10BF0DFEC07F00C
:10129000880EF6EC07F0E8CF00F1890EF6EC07F0C7
:1012A000E8CF01F100C140F601C141F602C142F6AA
:1012B00003C143F6D9EC34F062EC2FF0200EF6ECCB
:1012C00007F0E8CF2FF505012F51FF0AD8A470EFE2
:1012D00009F02F6B200E0C6E2FC50BF0DFEC07F022
:1012E0000501010E306F3C0E316F250EF6EC07F054
:1012F000E8CF00F1260EF6EC07F0E8CF01F1270E5B
:10130000F6EC07F0E8CF02F1280EF6EC07F0E8CF94
:1013100003F1010103AFA7EF09F0F2EC2AF0250E6B
:101320000C6E00C10BF0DFEC07F0260E0C6E01C155
:101330000BF0DFEC07F0270E0C6E02C10BF0DFECB8
:1013400007F0280E0C6E03C10BF0DFEC07F000C1B4
:1013500053F501C154F502C155F503C156F500C15D
:1013600057F501C158F502C159F503C15AF5290EC7
:10137000F6EC07F0E8CF5BF505015C515B5DD8A0AA
:101380005BC55CF505012F51020A0EE181B8D4EF6F
:1013900009F005015C2FD1EF09F05BC55CF5D4EFD6
:1013A00009F081BA18EF35F0210EF6EC07F0E8CF1E
:1013B00000F1220EF6EC07F0E8CF01F1230EF6EC77
:1013C00007F0E8CF02F1240EF6EC07F0E8CF03F1C6
:1013D000010103AF1AEF0AF0F2EC2AF0210E0C6EB5
:1013E00000C10BF0DFEC07F0220E0C6E01C10BF018
:1013F000DFEC07F0230E0C6E02C10BF0DFEC07F000
:10140000240E0C6E03C10BF0DFEC07F0210EF6EC9E
:1014100007F0E8CF00F1220EF6EC07F0E8CF01F17B
:10142000230EF6EC07F0E8CF02F1240EF6EC07F0FD
:10143000E8CF03F100C15DF501C15EF502C15FF5C2
:1014400003C160F599EC2EF05BEC2DF0ABEC2CF0C9
:1014500005012F51030A12E005012F51040A1DE076
:1014600005012F51050A24E005012F51060A32E03B
:1014700005012F51070A38E07DEF0AF0ACC500F1F5
:1014800001010F0E001701010051000A36E00101B1
:101490000051050A32E07AEF0AF0ACC500F1010113
:1014A0000F0E001701010051000A27E07AEF0AF041
:1014B0000501AC51000A21E00501AC51150A1DE0FF
:1014C0000501AC51300A19E00501AC51450A15E09F
:1014D0007AEF0AF00501AC51000A0FE00501AC51AA
:1014E000300A0BE07AEF0AF00501AC51000A05E082
:1014F0007AEF0AF081BA18EF35F056EC2CF007902D
:101500000001F28EF28C07B053EF26F00FB032EFED
:1015100021F00FB8F6EF1AF00301805181197F0B0B
:10152000D8B453EF26F013EE00F081517F0BE12683
:10153000812BE7CFE8FFE00BD8B453EF26F023EE82
:1015400082F0C2513F0BD926E7CFDFFFC22BDF501D
:10155000780AD8A453EF26F007808EC100F18FC11E
:1015600001F190C102F191C103F10101040E046F78
:10157000000E056F000E066F000E076FF7EC29F0E6
:1015800000AFCCEF0AF00101030E8E6F000E8F6FDB
:10159000000E906F000E916F03018251720AD8B451
:1015A00032EF21F08251520AD8B432EF21F0825149
:1015B000750AD8B432EF21F08251630AD8B40DEF26
:1015C00023F08251690AD8B4EDEF1DF082517A0AF6
:1015D000D8B400EF1FF08251490AD8B48CEF1DF047
:1015E0008251500AD8B4AAEF1CF08251700AD8B4C4
:1015F000EDEF1CF08251540AD8B418EF1DF082515F
:10160000740AD8B45EEF1DF082516D0AD8B438EF79
:101610000BF082514D0AD8B451EF0BF08251730A8E
:10162000D8B462EF20F08251530AD8B4C7EF20F04B
:1016300082514C0AD8B4B4EF12F08251760AD8B471
:10164000E0EF0BF044EF23F0040114EE00F08051C2
:101650007F0BE12682C4E7FF802B120004010D0EF0
:10166000826F24EC0BF00A0E826F24EC0BF0120058
:1016700004016D0E826F24EC0BF003018351300ADC
:10168000D8B490EF0BF003018351310AD8B4A3EF23
:101690000BF003018351320AD8B4B6EF0BF044EFDC
:1016A00023F004014D0E826F24EC0BF033EC2BF091
:1016B00084C331F185C332F186C333F10101296B53
:1016C00040EC2BF0B7EC2AF003018351300AD8B478
:1016D00078EF0BF003018351310AD8B480EF0BF09F
:1016E00003018351320AD8B488EF0BF044EF23F0A2
:1016F000FD0E0C6E00C10BF0DFEC07F090EF0BF06D
:10170000FE0E0C6E00C10BF0DFEC07F0A3EF0BF048
:10171000FF0E0C6E00C10BF0DFEC07F0B6EF0BF024
:101720000401300E826F24EC0BF004012C0E826F4A
:1017300024EC0BF0F2EC2AF0FD0EF6EC07F0E8CF0B
:1017400000F1C7EF0BF00401310E826F24EC0BF0B7
:1017500004012C0E826F24EC0BF0F2EC2AF0FE0E4A
:10176000F6EC07F0E8CF00F1C7EF0BF00401320E02
:10177000826F24EC0BF0F2EC2AF004012C0E826F45
:1017800024EC0BF0FF0EF6EC07F0E8CF00F195EC3F
:101790002AF031C182F40401300E822724EC0BF0D0
:1017A00032C182F40401300E822724EC0BF033C1E5
:1017B00082F40401300E822724EC0BF042EF23F078
:1017C00003018351300AD8B485EF0DF00301835132
:1017D000310AD8B4BCEF0DF003018351320AD8B4FA
:1017E00071EF0FF003018351330AD8B426EF11F0E3
:1017F00003018351340AD8B4CCEF11F003018351B3
:10180000730AD8B467EF0CF003018351760AD8B499
:1018100069EF0CF003018351740AD8B454EF0CF053
:1018200003018351540AD8B419EF0CF0D8A444EF43
:1018300023F00401760E826F24EC0BF00401540EA9
:10184000826F24EC0BF007840001880E0C6E33ECE1
:101850002BF02981030184512D0AD8B432EF0CF00A
:101860000101299185C32FF186C330F187C331F17E
:1018700088C332F189C333F140EC2BF0B7EC2AF086
:1018800000C10BF0DFEC07F001C10BF0DFEC07F05B
:10189000880EF6EC07F0E8CF40F6890EF6EC07F07C
:1018A000E8CF41F65FEF0CF00401760E826F24EC76
:1018B0000BF00401740E826F24EC0BF0078400011E
:1018C000880E0C6EFDEC07F0079457EF1BF067ECE9
:1018D0000CF00401760E826F24EC0BF00401760EFE
:1018E000826F24EC0BF007846FEC27F004012C0EC0
:1018F000826F24EC0BF00101036B026B3BC601F11C
:101900003AC600F101AF8AEF0CF00101FF0E026F41
:10191000FF0E036F95EC2AF0296791EF0CF096EF1C
:101920000CF004012D0E826F24EC0BF02FC182F419
:101930000401300E822724EC0BF030C182F4040144
:10194000300E822724EC0BF031C182F40401300EFA
:10195000822724EC0BF032C182F40401300E82277E
:1019600024EC0BF033C182F40401300E822724EC06
:101970000BF004012C0E826F24EC0BF00101036BC1
:10198000026B3DC601F13CC600F101AFCDEF0CF09A
:101990000101FF0E026FFF0E036F95EC2AF029671D
:1019A000D4EF0CF0D9EF0CF004012D0E826F24EC73
:1019B0000BF02FC182F40401300E822724EC0BF0CF
:1019C00030C182F40401300E822724EC0BF031C1C7
:1019D00082F40401300E822724EC0BF032C182F431
:1019E0000401300E822724EC0BF033C182F4040191
:1019F000300E822724EC0BF004012C0E826F24ECB5
:101A00000BF00101036B026B3FC601F13EC600F112
:101A100001AF10EF0DF00101FF0E026FFF0E036F1B
:101A200095EC2AF0296717EF0DF01CEF0DF004017B
:101A30002D0E826F24EC0BF02FC182F40401300EC6
:101A4000822724EC0BF030C182F40401300E82278F
:101A500024EC0BF031C182F40401300E822724EC17
:101A60000BF032C182F40401300E822724EC0BF01B
:101A700033C182F40401300E822724EC0BF0040100
:101A80002C0E826F24EC0BF00101036B026B37C646
:101A900001F136C600F101AF53EF0DF00101FF0E69
:101AA000026FFF0E036F95EC2AF029675AEF0DF0D5
:101AB0005FEF0DF004012D0E826F24EC0BF02FC1AF
:101AC00082F40401300E822724EC0BF030C182F442
:101AD0000401300E822724EC0BF031C182F40401A2
:101AE000300E822724EC0BF032C182F40401300E58
:101AF000822724EC0BF033C182F40401300E8227DC
:101B000024EC0BF0079457EF1BF00401760E826F64
:101B100024EC0BF00401300E826F24EC0BF0040176
:101B20002C0E826F24EC0BF060EC2BF0F2EC2AF020
:101B300000C600F101C601F195EC2AF030C182F433
:101B40000401300E822724EC0BF031C182F4040131
:101B5000300E822724EC0BF032C182F40401300EE7
:101B6000822724EC0BF033C182F40401300E82276B
:101B700024EC0BF057EF1BF00401760E826F24EC7F
:101B80000BF00401310E826F24EC0BF0078401018D
:101B9000036B026B02C600F103C601F101AFD5EF82
:101BA0000DF0FF0E026FFF0E036F0101076B066B56
:101BB00004C604F105C605F105AFE3EF0DF0FF0E15
:101BC000066FFF0E076FFCEC29F00101076B066B37
:101BD00006C604F107C605F105AFF3EF0DF0FF0EE1
:101BE000066FFF0E076FFCEC29F00101076B066B17
:101BF00008C604F109C605F105AF03EF0EF0FF0EAC
:101C0000066FFF0E076FFCEC29F0D890010103333B
:101C1000023301330033D89001010333023301331F
:101C2000003304012C0E826F24EC0BF00101036BD6
:101C3000026B01C101F100C100F101AF25EF0EF00F
:101C40000101FF0E026FFF0E036F95EC2AF029676A
:101C50002CEF0EF031EF0EF004012D0E826F24EC0C
:101C60000BF02FC182F40401300E822724EC0BF01C
:101C700030C182F40401300E822724EC0BF031C114
:101C800082F40401300E822724EC0BF032C182F47E
:101C90000401300E822724EC0BF033C182F40401DE
:101CA000300E822724EC0BF00101036B026B0AC695
:101CB00000F10BC601F101AF62EF0EF0FF0E026FF3
:101CC000FF0E036F0101076B066B0CC604F10DC616
:101CD00005F105AF70EF0EF0FF0E066FFF0E076FF8
:101CE000FCEC29F00101076B066B0EC604F10FC670
:101CF00005F105AF80EF0EF0FF0E066FFF0E076FC8
:101D0000FCEC29F00101076B066B10C604F111C64B
:101D100005F105AF90EF0EF0FF0E066FFF0E076F97
:101D2000FCEC29F0D8900101033302330133003376
:101D3000D8900101033302330133003304012C0E28
:101D4000826F24EC0BF00101036B026B01C101F106
:101D500000C100F101AFB2EF0EF00101FF0E026F02
:101D6000FF0E036F95EC2AF02967B9EF0EF0BEEF76
:101D70000EF004012D0E826F24EC0BF02FC182F4C3
:101D80000401300E822724EC0BF030C182F40401F0
:101D9000300E822724EC0BF031C182F40401300EA6
:101DA000822724EC0BF032C182F40401300E82272A
:101DB00024EC0BF033C182F40401300E822724ECB2
:101DC0000BF00101036B026B12C600F113C601F1A7
:101DD00001AFEFEF0EF0FF0E026FFF0E036F010178
:101DE000076B066B14C604F115C605F105AFFDEFD0
:101DF0000EF0FF0E066FFF0E076FFCEC29F00101DD
:101E0000076B066B16C604F117C605F105AF0DEF9B
:101E10000FF0FF0E066FFF0E076FFCEC29F00101BB
:101E2000076B066B18C604F119C605F105AF1DEF67
:101E30000FF0FF0E066FFF0E076FFCEC29F0D89035
:101E400001010333023301330033D890010103331E
:101E500002330133003304012C0E826F24EC0BF0AB
:101E60000101036B026B01C101F100C100F101AF7F
:101E70003FEF0FF00101FF0E026FFF0E036F95ECB5
:101E80002AF0296746EF0FF04BEF0FF004012D0EFB
:101E9000826F24EC0BF02FC182F40401300E8227F4
:101EA00024EC0BF030C182F40401300E822724ECC4
:101EB0000BF031C182F40401300E822724EC0BF0C8
:101EC00032C182F40401300E822724EC0BF033C1BE
:101ED00082F40401300E822724EC0BF0079457EFB4
:101EE0001BF00401760E826F24EC0BF00401320E1D
:101EF000826F24EC0BF007840101036B026B1AC69E
:101F000000F11BC601F101AF8AEF0FF0FF0E026F67
:101F1000FF0E036F0101076B066B1CC604F11DC6A3
:101F200005F105AF98EF0FF0FF0E066FFF0E076F7C
:101F3000FCEC29F00101076B066B1EC604F11FC6FD
:101F400005F105AFA8EF0FF0FF0E066FFF0E076F4C
:101F5000FCEC29F00101076B066B20C604F121C6D9
:101F600005F105AFB8EF0FF0FF0E066FFF0E076F1C
:101F7000FCEC29F0D8900101033302330133003324
:101F8000D8900101033302330133003304012C0ED6
:101F9000826F24EC0BF00101036B026B01C101F1B4
:101FA00000C100F101AFDAEF0FF00101FF0E026F87
:101FB000FF0E036F95EC2AF02967E1EF0FF0E6EFD3
:101FC0000FF004012D0E826F24EC0BF02FC182F470
:101FD0000401300E822724EC0BF030C182F404019E
:101FE000300E822724EC0BF031C182F40401300E54
:101FF000822724EC0BF032C182F40401300E8227D8
:1020000024EC0BF033C182F40401300E822724EC5F
:102010000BF00101036B026B22C600F123C601F134
:1020200001AF17EF10F0FF0E026FFF0E036F0101FB
:10203000076B066B24C604F125C605F105AF25EF35
:1020400010F0FF0E066FFF0E076FFCEC29F0010188
:10205000076B066B26C604F127C605F105AF35EF01
:1020600010F0FF0E066FFF0E076FFCEC29F0010168
:10207000076B066B28C604F129C605F105AF45EFCD
:1020800010F0FF0E066FFF0E076FFCEC29F0D890E2
:1020900001010333023301330033D89001010333CC
:1020A00002330133003304012C0E826F24EC0BF059
:1020B0000101036B026B01C101F100C100F101AF2D
:1020C00067EF10F00101FF0E026FFF0E036F95EC3A
:1020D0002AF029676EEF10F073EF10F004012D0E57
:1020E000826F24EC0BF02FC182F40401300E8227A2
:1020F00024EC0BF030C182F40401300E822724EC72
:102100000BF031C182F40401300E822724EC0BF075
:1021100032C182F40401300E822724EC0BF033C16B
:1021200082F40401300E822724EC0BF00101036BD2
:10213000026B2AC600F12BC601F101AFA4EF10F02B
:10214000FF0E026FFF0E036F0101076B066B2CC6BB
:1021500004F12DC605F105AFB2EF10F0FF0E066FCA
:10216000FF0E076FFCEC29F00101076B066B2EC612
:1021700004F12FC605F105AFC2EF10F0FF0E066F98
:10218000FF0E076FFCEC29F00101076B066B30C6F0
:1021900004F131C605F105AFD2EF10F0FF0E066F66
:1021A000FF0E076FFCEC29F0D890010103330233D6
:1021B00001330033D890010103330233013300337C
:1021C00004012C0E826F24EC0BF00101036B026BF7
:1021D00001C101F100C100F101AFF4EF10F0010104
:1021E000FF0E026FFF0E036F95EC2AF02967FBEFDD
:1021F00010F000EF11F004012D0E826F24EC0BF0B3
:102200002FC182F40401300E822724EC0BF030C180
:1022100082F40401300E822724EC0BF031C182F4E9
:102220000401300E822724EC0BF032C182F4040149
:10223000300E822724EC0BF033C182F40401300EFF
:10224000822724EC0BF0079457EF1BF00401760E65
:10225000826F24EC0BF00401330E826F24EC0BF040
:1022600004012C0E826F24EC0BF085C382F424EC65
:102270000BF0640E0D6E03018551320A02E16A0E05
:102280000D6E03018551330A02E1700E0D6E0301DC
:102290008551340A02E1760E0D6E03018551350A2F
:1022A00002E17C0E0D6E03018551360A02E1820EB9
:1022B0000D6E03018651780A65E00DC00CF033EC19
:1022C0002BF02981030187512D0AD8B46AEF11F050
:1022D0000101299188C32FF189C330F18AC331F1FB
:1022E0008BC332F18CC333F140EC2BF0B7EC2AF006
:1022F00000C10BF0DFEC07F001C10BF0DFEC07F0E1
:1023000033EC2BF0298103018E512D0AD8B48BEFC9
:1023100011F0010129918FC32FF190C330F191C3C6
:1023200031F192C332F193C333F140EC2BF0B7ECAF
:102330002AF000C10BF0DFEC07F001C10BF0DFEC7D
:1023400007F033EC2BF02981030195512D0AD8B405
:10235000ACEF11F00101299196C32FF197C330F131
:1023600098C331F199C332F19AC333F140EC2BF0A9
:10237000B7EC2AF000C10BF0DFEC07F001C10BF065
:10238000DFEC07F00DC00CF0FDEC07F0FDEC07F002
:10239000FDEC07F057EF1BF00401760E826F24EC82
:1023A0000BF00401340E826F24EC0BF00301845116
:1023B000780AD8B4A4EF12F03E0E0C6E33EC2BF07A
:1023C0002981030185512D0AD8B4E9EF11F00101EB
:1023D000299186C32FF187C330F188C331F189C3B6
:1023E00032F18AC333F140EC2BF0B7EC2AF000C194
:1023F0000BF0DFEC07F001C10BF0DFEC07F033EC82
:102400002BF0298103018C512D0AD8B40AEF12F068
:10241000010129918DC32FF18EC330F18FC331F1AA
:1024200090C332F191C333F140EC2BF0B7EC2AF0BA
:1024300000C10BF0DFEC07F001C10BF0DFEC07F09F
:1024400033EC2BF02981030193512D0AD8B42BEFE3
:1024500012F00101299194C32FF195C330F196C375
:1024600031F197C332F198C333F140EC2BF0B7EC64
:102470002AF000C10BF0DFEC07F001C10BF0DFEC3C
:1024800007F033EC2BF0298103019A512D0AD8B4BF
:102490004CEF12F0010129919BC32FF19CC330F145
:1024A0009DC331F19EC332F19FC333F140EC2BF059
:1024B000B7EC2AF000C10BF0DFEC07F001C10BF024
:1024C000DFEC07F033EC2BF029810301A1512D0A39
:1024D000D8B46DEF12F001012991A2C32FF1A3C36B
:1024E00030F1A4C331F1A5C332F1A6C333F140ECFE
:1024F0002BF0B7EC2AF000C10BF0DFEC07F001C1C4
:102500000BF0DFEC07F033EC2BF029810301A8512D
:102510002D0AD8B48EEF12F001012991A9C32FF131
:10252000AAC330F1ABC331F1ACC332F1ADC333F167
:1025300040EC2BF0B7EC2AF000C10BF0DFEC07F019
:1025400001C10BF0DFEC07F03E0E0C6EFDEC07F066
:10255000FDEC07F0FDEC07F0FDEC07F0FDEC07F0FB
:10256000FDEC07F057EF1BF003018351300AD8B49C
:1025700019EF16F003018351310AD8B427EF17F091
:1025800003018351320AD8B495EF17F00301835148
:10259000330AD8B4A5EF17F003018351340AD8B435
:1025A000B5EF17F003018351350AD8B4FBEF1AF0E9
:1025B00003018351360AD8B429EF1BF0030183517C
:1025C000370AD8B47BEF15F003018351460AD8B41B
:1025D0004FEF1AF0030183514D0AD8B4F4EF13F012
:1025E000030183516D0AD8B40EEF14F00301835137
:1025F0005A0AD8B4A1EF16F003018351490AD8B49E
:1026000029EF1CF003018351500AD8B45BEF1BF093
:1026100003018351540AD8B4D4EF1BF00301835152
:10262000630AD8B42EEF14F003018351430AD8B4DF
:1026300026EF15F003018351730AD8B42CEF14F080
:1026400003018351610AD8B441EF13F003018351B0
:10265000650AD8B469EF16F003018351450AD8B46E
:1026600077EF16F003018351620AD8B485EF16F0B4
:1026700003018351420AD8B493EF16F0D8A444EF73
:1026800023F004014C0E826F24EC0BF00401610E68
:10269000826F24EC0BF05BEC2DF004012C0E826FAA
:1026A00024EC0BF0F2EC2AF0ABC500F1010195EC43
:1026B0002AF031C182F40401300E822724EC0BF0A1
:1026C00032C182F40401300E822724EC0BF033C1B6
:1026D00082F40401300E822724EC0BF004012C0E4E
:1026E000826F24EC0BF0F2EC2AF0ACC500F1010192
:1026F00095EC2AF031C182F40401300E822724ECDB
:102700000BF032C182F40401300E822724EC0BF06E
:1027100033C182F40401300E822724EC0BF0040153
:102720002C0E826F24EC0BF0F2EC2AF0ADC500F118
:10273000010195EC2AF031C182F40401300E8227A8
:1027400024EC0BF032C182F40401300E822724EC19
:102750000BF033C182F40401300E822724EC0BF01D
:1027600004012C0E826F24EC0BF0F2EC2AF0AEC5C3
:1027700000F1010195EC2AF031C182F40401300E20
:10278000822724EC0BF032C182F40401300E822740
:1027900024EC0BF033C182F40401300E822724ECC8
:1027A0000BF004012C0E826F24EC0BF0F2EC2AF0FB
:1027B000B3C500F1010195EC2AF031C182F40401A6
:1027C000300E822724EC0BF032C182F40401300E6B
:1027D000822724EC0BF033C182F40401300E8227EF
:1027E00024EC0BF057EF1BF033EC2BF084C333F1E8
:1027F00040EC2BF0B7EC2AF0200E0C6E00C10BF071
:10280000DFEC07F000C12FF505012F51000A06E0AB
:1028100005012F51010A02E001EC2EF004014C0EDB
:10282000826F24EC0BF004014D0E826F24EC0BF050
:1028300004012C0E826F24EC0BF0F2EC2AF02FC571
:1028400000F195EC2AF033C182F40401300E8227A6
:1028500024EC0BF057EF1BF018EF35F004014C0E91
:10286000826F24EC0BF00401630E826F24EC0BF0FA
:10287000ABEC2CF004012C0E826F24EC0BF043EC3B
:1028800014F057EF1BF0F2EC2AF0B1C500F1010192
:10289000003B0F0E001795EC2AF033C182F40401BF
:1028A000300E822724EC0BF0B1C500F101010F0EB0
:1028B0000101001795EC2AF033C182F40401300EB7
:1028C000822724EC0BF004012D0E826F24EC0BF018
:1028D000B0C500F10101003B0F0E001795EC2AF086
:1028E00033C182F40401300E822724EC0BF0B0C512
:1028F00000F101010F0E0101001795EC2AF033C120
:1029000082F40401300E822724EC0BF004012D0E1A
:10291000826F24EC0BF0AFC500F10101003B0F0EFC
:10292000001795EC2AF033C182F40401300E82279F
:1029300024EC0BF0AFC500F101010F0E01010017EF
:1029400095EC2AF033C182F40401300E822724EC86
:102950000BF00401200E826F24EC0BF0AEC500F1E9
:102960000F0E0101001795EC2AF033C182F4040127
:10297000300E822724EC0BF00401200E826F24EC31
:102980000BF0ADC500F101010101003B0F0E001776
:1029900095EC2AF033C182F40401300E822724EC36
:1029A0000BF0ADC500F101010F0E0101001795EC10
:1029B0002AF033C182F40401300E822724EC0BF09C
:1029C00004013A0E826F24EC0BF0ACC500F101015A
:1029D000003B0F0E001795EC2AF033C182F404017E
:1029E000300E822724EC0BF0ACC500F101010F0E74
:1029F0000101001795EC2AF033C182F40401300E76
:102A0000822724EC0BF004013A0E826F24EC0BF0C9
:102A1000ABC500F10101003B0F0E001795EC2AF049
:102A200033C182F40401300E822724EC0BF0ABC5D5
:102A300000F101010F0E001795EC2AF033C182F46A
:102A40000401300E822724EC0BF0120084C3E8FF4F
:102A50000F0BE83AE8CFB1F585C3E8FF0F0B05018E
:102A6000B11387C3E8FF0F0BE83AE8CFB0F588C38E
:102A7000E8FF0F0B0501B0138AC3E8FF0F0BE83A1C
:102A8000E8CFAFF58BC3E8FF0F0B0501AF138DC384
:102A9000E8FF0F0BE8CFAEF58FC3E8FF0F0BE83A66
:102AA000E8CFADF590C3E8FF0F0B0501AD1392C35E
:102AB000E8FF0F0BE83AE8CFACF593C3E8FF0F0B44
:102AC0000501AC1395C3E8FF0F0BE83AE8CFABF56F
:102AD00096C3E8FF0F0B0501AB130AEC2DF00401C0
:102AE0004C0E826F24EC0BF00401430E826F24EC39
:102AF0000BF038EF14F0078404014C0E826F24ECC5
:102B00000BF00401370E826F24EC0BF004012C0E45
:102B1000826F24EC0BF005012E51130A06E005012B
:102B20002E51170A0DE016EF16F00101000E006F8E
:102B3000000E016F100E026F000E036FA9EF15F06B
:102B40000101000E006F000E016F000E026F010EFA
:102B5000036F95EC2AF02AC182F40401300E82271B
:102B600024EC0BF02BC182F40401300E822724ECFC
:102B70000BF02CC182F40401300E822724EC0BF000
:102B80002DC182F40401300E822724EC0BF02EC1FB
:102B900082F40401300E822724EC0BF02FC182F462
:102BA0000401300E822724EC0BF030C182F40401C2
:102BB000300E822724EC0BF031C182F40401300E78
:102BC000822724EC0BF032C182F40401300E8227FC
:102BD00024EC0BF033C182F40401300E822724EC84
:102BE0000BF004012C0E826F24EC0BF00101200E7F
:102BF000006F000E016F000E026F000E036F95EC68
:102C00002AF031C182F40401300E822724EC0BF04B
:102C100032C182F40401300E822724EC0BF033C160
:102C200082F40401300E822724EC0BF0079457EF56
:102C30001BF00784D9EC34F0F2EC2AF02DC500F13A
:102C400095EC2AF004014C0E826F24EC0BF0040189
:102C5000300E826F24EC0BF004012C0E826F24ECFA
:102C60000BF031C182F40401300E822724EC0BF00A
:102C700032C182F40401300E822724EC0BF033C100
:102C800082F40401300E822724EC0BF004012C0E98
:102C9000826F24EC0BF0F2EC2AF02EC500F195ECDB
:102CA0002AF031C182F40401300E822724EC0BF0AB
:102CB00032C182F40401300E822724EC0BF033C1C0
:102CC00082F40401300E822724EC0BF0079457EFB6
:102CD0001BF004014C0E826F24EC0BF00401650E16
:102CE000826F24EC0BF0EAEC2EF057EF1BF004019E
:102CF0004C0E826F24EC0BF00401450E826F24EC25
:102D00000BF007EC2FF057EF1BF004014C0E826F15
:102D100024EC0BF00401620E826F24EC0BF041EC0A
:102D20002FF057EF1BF004014C0E826F24EC0BF0D8
:102D30000401420E826F24EC0BF024EC2FF057EFCD
:102D40001BF004014C0E826F24EC0BF004015A0EB0
:102D5000826F24EC0BF004012C0E826F24EC0BF03C
:102D6000D9EC34F0F2EC2AF005012E51130A06E0FA
:102D700005012E51170A0DE0D2EF16F00101000EE9
:102D8000006F000E016F100E026F000E036FD2EF86
:102D900016F00101000E006F000E016F000E026FB1
:102DA000010E036F0101200E046F000E056F000E6F
:102DB000066F000E076F28EC2AF095EC2AF02AC166
:102DC00082F40401300E822724EC0BF02BC182F434
:102DD0000401300E822724EC0BF02CC182F4040194
:102DE000300E822724EC0BF02DC182F40401300E4A
:102DF000822724EC0BF02EC182F40401300E8227CE
:102E000024EC0BF02FC182F40401300E822724EC55
:102E10000BF030C182F40401300E822724EC0BF059
:102E200031C182F40401300E822724EC0BF032C150
:102E300082F40401300E822724EC0BF033C182F4BB
:102E40000401300E822724EC0BF057EF1BF00784AF
:102E500004014C0E826F24EC0BF00401310E826FE2
:102E600024EC0BF004012C0E826F24EC0BF025C532
:102E700000F126C501F127C502F128C503F10101C2
:102E8000200E046F000E056F000E066F000E076F18
:102E900028EC2AF095EC2AF02AC182F40401300EC5
:102EA000822724EC0BF02BC182F40401300E822720
:102EB00024EC0BF02CC182F40401300E822724ECA8
:102EC0000BF02DC182F40401300E822724EC0BF0AC
:102ED0002EC182F40401300E822724EC0BF02FC1A6
:102EE00082F40401300E822724EC0BF030C182F40E
:102EF0000401300E822724EC0BF031C182F404016E
:102F0000300E822724EC0BF032C182F40401300E23
:102F1000822724EC0BF033C182F40401300E8227A7
:102F200024EC0BF0079457EF1BF0078404014C0EC0
:102F3000826F24EC0BF00401320E826F24EC0BF054
:102F400037EC31F0079457EF1BF0078404014C0E67
:102F5000826F24EC0BF00401330E826F24EC0BF033
:102F600094EC31F0079432EF17F0078404014C0E13
:102F7000826F24EC0BF00401340E826F24EC0BF012
:102F800004012C0E826F24EC0BF033EC2BF084C385
:102F90002AF185C32BF186C32CF187C32DF188C399
:102FA0002EF189C32FF18AC330F18BC331F18CC369
:102FB00032F18DC333F10101296B40EC2BF0B7ECFA
:102FC0002AF0200E046F000E056F000E066F000E33
:102FD000076F08EC2AF000C121F501C122F502C1FA
:102FE00023F503C124F58CEC34F034C5ABF535C5BD
:102FF000ACF536C5ADF537C5AEF538C5AFF539C555
:10300000B0F53AC5B1F543EC14F004012C0E826F13
:1030100024EC0BF03BC500F13CC501F13DC502F1CC
:103020003EC503F10101000E046F000E056F010E95
:10303000066F000E076F28EC2AF095EC2AF029673E
:1030400024EF18F029EF18F004012D0E826F24EC04
:103050000BF030C182F40401300E822724EC0BF017
:1030600031C182F40401300E822724EC0BF00401FC
:103070002E0E826F24EC0BF032C182F40401300E6C
:10308000822724EC0BF033C182F40401300E822736
:1030900024EC0BF004012C0E826F24EC0BF0F2EC0C
:1030A0002AF03FC500F140C501F16EEC24F00401A7
:1030B0002C0E826F24EC0BF0F2EC2AF041C500F1EB
:1030C00095EC2AF031C182F40401300E822724EC01
:1030D0000BF032C182F40401300E822724EC0BF095
:1030E00033C182F40401300E822724EC0BF004017A
:1030F0002C0E826F24EC0BF00101036B026B48C5B0
:1031000001F147C500F101AF8BEF18F00101FF0E8F
:10311000026FFF0E036F95EC2AF0296792EF18F00B
:1031200097EF18F004012D0E826F24EC0BF02FC1E5
:1031300082F40401300E822724EC0BF030C182F4BB
:103140000401300E822724EC0BF031C182F404011B
:10315000300E822724EC0BF032C182F40401300ED1
:10316000822724EC0BF033C182F40401300E822755
:1031700024EC0BF004012C0E826F24EC0BF0010107
:10318000036B026B4AC501F149C500F101AFCEEFF7
:1031900018F00101FF0E026FFF0E036F95EC2AF08D
:1031A0002967D5EF18F0DAEF18F004012D0E826FC1
:1031B00024EC0BF02FC182F40401300E822724ECA2
:1031C0000BF030C182F40401300E822724EC0BF0A6
:1031D00031C182F40401300E822724EC0BF032C19D
:1031E00082F40401300E822724EC0BF033C182F408
:1031F0000401300E822724EC0BF004012C0E826FA8
:1032000024EC0BF00101036B026B4CC501F14BC5C3
:1032100000F101AF11EF19F00101FF0E026FFF0E77
:10322000036F95EC2AF0296718EF19F01DEF19F0DC
:1032300004012D0E826F24EC0BF02FC182F40401E7
:10324000300E822724EC0BF030C182F40401300EE2
:10325000822724EC0BF031C182F40401300E822766
:1032600024EC0BF032C182F40401300E822724ECEE
:103270000BF033C182F40401300E822724EC0BF0F2
:1032800004012C0E826F24EC0BF00101036B026B26
:103290004EC501F14DC500F101AF54EF19F0010128
:1032A000FF0E026FFF0E036F95EC2AF029675BEFAC
:1032B00019F060EF19F004012D0E826F24EC0BF071
:1032C0002FC182F40401300E822724EC0BF030C1B0
:1032D00082F40401300E822724EC0BF031C182F419
:1032E0000401300E822724EC0BF032C182F4040179
:1032F000300E822724EC0BF033C182F40401300E2F
:10330000822724EC0BF004012C0E826F24EC0BF0CE
:103310000101036B026B50C501F14FC500F101AF14
:1033200097EF19F00101FF0E026FFF0E036F95EC8E
:103330002AF029679EEF19F0A3EF19F004012D0E72
:10334000826F24EC0BF02FC182F40401300E82272F
:1033500024EC0BF030C182F40401300E822724ECFF
:103360000BF031C182F40401300E822724EC0BF003
:1033700032C182F40401300E822724EC0BF033C1F9
:1033800082F40401300E822724EC0BF004012C0E91
:10339000826F24EC0BF00101036B026B52C501F14B
:1033A00051C500F101AFDAEF19F00101FF0E026F14
:1033B000FF0E036F95EC2AF02967E1EF19F0E6EFB5
:1033C00019F004012D0E826F24EC0BF02FC182F452
:1033D0000401300E822724EC0BF030C182F404018A
:1033E000300E822724EC0BF031C182F40401300E40
:1033F000822724EC0BF032C182F40401300E8227C4
:1034000024EC0BF033C182F40401300E822724EC4B
:103410000BF004012C0E826F24EC0BF00101036B06
:10342000026B46C501F145C500F101AF1DEF1AF071
:103430000101FF0E026FFF0E036F95EC2AF0296762
:1034400024EF1AF029EF1AF004012D0E826F24ECFC
:103450000BF02FC182F40401300E822724EC0BF014
:1034600030C182F40401300E822724EC0BF031C10C
:1034700082F40401300E822724EC0BF032C182F476
:103480000401300E822724EC0BF033C182F40401D6
:10349000300E822724EC0BF0079457EF1BF033EC2F
:1034A0002BF085C32AF186C32BF187C32CF188C387
:1034B0002DF189C32EF18AC32FF18BC330F18CC358
:1034C00031F18DC332F18EC333F10101296B40EC30
:1034D0002BF0B7EC2AF00101010E046F000E056F0E
:1034E000000E066F000E076FF7EC29F0100E046F48
:1034F000000E056F000E066F000E076F08EC2AF035
:1035000000C129F501C12AF502C12BF503C12CF533
:10351000C0EC30F004014C0E826F24EC0BF004017F
:10352000460E826F24EC0BF004012C0E826F24EC0B
:103530000BF025C500F126C501F127C502F128C50C
:1035400003F10101100E046F000E056F000E066FEF
:10355000000E076F28EC2AF095EC2AF02AC182F4BD
:103560000401300E822724EC0BF02BC182F40401FD
:10357000300E822724EC0BF02CC182F40401300EB3
:10358000822724EC0BF02DC182F40401300E822737
:1035900024EC0BF02EC182F40401300E822724ECBF
:1035A0000BF02FC182F40401300E822724EC0BF0C3
:1035B00030C182F40401300E822724EC0BF031C1BB
:1035C00082F40401300E822724EC0BF032C182F425
:1035D0000401300E822724EC0BF033C182F4040185
:1035E000300E822724EC0BF057EF1BF00F9894EC71
:1035F00031F044EF23F004014C0E826F24EC0BF009
:103600000401350E826F24EC0BF004012C0E826F46
:1036100024EC0BF0F2EC2AF00784B5C500F1079416
:1036200095EC2AF031C182F40401300E822724EC9B
:103630000BF032C182F40401300E822724EC0BF02F
:1036400033C182F40401300E822724EC0BF057EFD3
:103650001BF057EC31F0F2EC2AF033C500F195EC99
:103660002AF004014C0E826F24EC0BF00401360E9C
:10367000826F24EC0BF004012C0E826F24EC0BF013
:1036800031C182F40401300E822724EC0BF032C1E8
:1036900082F40401300E822724EC0BF033C182F453
:1036A0000401300E822724EC0BF057EF1BF02EECB8
:1036B0000BF044EF23F004014C0E826F24EC0BF06E
:1036C0000401500E826F24EC0BF004012C0E826F6B
:1036D00024EC0BF085C32AF186C32BF187C32CF1B0
:1036E00088C32DF189C32EF18AC32FF18BC330F12A
:1036F0008CC331F18DC332F18EC333F1010140EC43
:103700002BF0B7EC2AF003018451530A0DE00301BA
:1037100084514D0A38E00401780E826F24EC0BF0DE
:103720002EEC0BF044EF23F00401530E826F24ECD7
:103730000BF0250E0C6E00C10BF0DFEC07F0260E2F
:103740000C6E01C10BF0DFEC07F0270E0C6E02C10E
:103750000BF0DFEC07F0280E0C6E03C10BF0DFEC72
:1037600007F000C153F501C154F502C155F503C17D
:1037700056F500C157F501C158F502C159F503C10D
:103780005AF538EF1CF004014D0E826F24EC0BF05B
:10379000290E0C6E00C10BF0DFEC07F000C15BF5E9
:1037A00000C15CF538EF1CF004014C0E826F24EC74
:1037B0000BF00401540E826F24EC0BF004012C0E6C
:1037C000826F24EC0BF084C32AF185C32BF186C3EE
:1037D0002CF187C32DF188C32EF189C32FF18AC341
:1037E00030F18BC331F18DC332F18EC333F101015E
:1037F00040EC2BF0B7EC2AF00101000E046F000E34
:10380000056F010E066F000E076F08EC2AF0210EFF
:103810000C6E00C10BF0DFEC07F0220E0C6E01C144
:103820000BF0DFEC07F0230E0C6E02C10BF0DFECA7
:1038300007F0240E0C6E03C10BF0DFEC07F000C1A3
:103840005DF501C15EF502C15FF503C160F538EFBA
:103850001CF004014C0E826F24EC0BF00401490EA5
:10386000826F24EC0BF004012C0E826F24EC0BF021
:10387000250EF6EC07F0E8CF00F1260EF6EC07F087
:10388000E8CF01F1270EF6EC07F0E8CF02F1280EA1
:10389000F6EC07F0E8CF03F195EC2AF078EC28F08D
:1038A0000401730E826F24EC0BF004012C0E826F66
:1038B00024EC0BF0F2EC2AF0290EF6EC07F0E8CF3E
:1038C00000F195EC2AF078EC28F00401730E826F79
:1038D00024EC0BF004012C0E826F24EC0BF057C586
:1038E00000F158C501F159C502F15AC503F195EC33
:1038F0002AF078EC28F00401730E826F24EC0BF0B0
:1039000004012C0E826F24EC0BF0F2EC2AF05CC563
:1039100000F195EC2AF078EC28F004016D0E826F2E
:1039200024EC0BF004012C0E826F24EC0BF05DC52F
:1039300000F15EC501F15FC502F160C503F15FEC06
:1039400023F004012C0E826F24EC0BF02EEC0BF014
:1039500044EF23F083C32AF184C32BF185C32CF1F8
:1039600086C32DF187C32EF188C32FF189C330F1AF
:103970008AC331F18BC332F18CC333F1010140ECC6
:103980002BF0B7EC2AF0160E0C6E00C10BF0DFEC3A
:1039900007F0170E0C6E01C10BF0DFEC07F0180EEC
:1039A0000C6E02C10BF0DFEC07F0190E0C6E03C1B8
:1039B0000BF0DFEC07F000C18AF101C18BF102C10D
:1039C0008CF103C18DF100C18EF101C18FF102C1F3
:1039D00090F103C191F18CEF1DF083C32AF184C3F0
:1039E0002BF185C32CF186C32DF187C32EF188C33B
:1039F0002FF189C330F18AC331F18BC332F18CC30B
:103A000033F1010140EC2BF0B7EC2AF000C18AF150
:103A100001C18BF102C18CF103C18DF100C18EF1A6
:103A200001C18FF102C190F103C191F18CEF1DF042
:103A300083C32AF184C32BF185C32CF186C32DF1F6
:103A400087C32EF188C32FF189C330F18AC331F1C6
:103A50008CC332F18DC333F1010140EC2BF0B7EC94
:103A60002AF00101000E046F000E056F010E066FB3
:103A7000000E076F08EC2AF01A0E0C6E00C10BF056
:103A8000DFEC07F01B0E0C6E01C10BF0DFEC07F052
:103A90001C0E0C6E02C10BF0DFEC07F01D0E0C6E5D
:103AA00003C10BF0DFEC07F000C192F101C193F10B
:103AB00002C194F103C195F18CEF1DF083C32AF18B
:103AC00084C32BF185C32CF186C32DF187C32EF15E
:103AD00088C32FF189C330F18AC331F18CC332F12D
:103AE0008DC333F1010140EC2BF0B7EC2AF001015A
:103AF000000E046F000E056F010E066F000E076FBB
:103B000008EC2AF000C192F101C193F102C194F1D5
:103B100003C195F18CEF1DF0160EF6EC07F0E8CF1F
:103B200000F1170EF6EC07F0E8CF01F1180EF6ECF5
:103B300007F0E8CF02F1190EF6EC07F0E8CF03F139
:103B400095EC2AF078EC28F00401730E826F24ECD7
:103B50000BF004012C0E826F24EC0BF08AC100F1F3
:103B60008BC101F18CC102F18DC103F195EC2AF0FA
:103B700078EC28F00401730E826F24EC0BF0040142
:103B80002C0E826F24EC0BF01A0EF6EC07F0E8CF47
:103B900000F11B0EF6EC07F0E8CF01F11C0EF6EC7D
:103BA00007F0E8CF02F11D0EF6EC07F0E8CF03F1C5
:103BB0005FEC23F004012C0E826F24EC0BF092C119
:103BC00000F193C101F194C102F195C103F15FECE1
:103BD00023F02EEC0BF044EF23F00401690E826F0A
:103BE00024EC0BF004012C0E826F24EC0BF001018D
:103BF000040E006F000E016F000E026F000E036FC7
:103C000095EC2AF02CC182F40401300E822724ECBA
:103C10000BF02DC182F40401300E822724EC0BF04E
:103C20002EC182F40401300E822724EC0BF02FC148
:103C300082F40401300E822724EC0BF030C182F4B0
:103C40000401300E822724EC0BF031C182F4040110
:103C5000300E822724EC0BF032C182F40401300EC6
:103C6000822724EC0BF033C182F40401300E82274A
:103C700024EC0BF004012C0E826F24EC0BF00101FC
:103C80000B0E006F000E016F000E026F000E036F2F
:103C900095EC2AF02CC182F40401300E822724EC2A
:103CA0000BF02DC182F40401300E822724EC0BF0BE
:103CB0002EC182F40401300E822724EC0BF02FC1B8
:103CC00082F40401300E822724EC0BF030C182F420
:103CD0000401300E822724EC0BF031C182F4040180
:103CE000300E822724EC0BF032C182F40401300E36
:103CF000822724EC0BF033C182F40401300E8227BA
:103D000024EC0BF004012C0E826F24EC0BF001016B
:103D1000230E006F000E016F000E026F000E036F86
:103D200095EC2AF02CC182F40401300E822724EC99
:103D30000BF02DC182F40401300E822724EC0BF02D
:103D40002EC182F40401300E822724EC0BF02FC127
:103D500082F40401300E822724EC0BF030C182F48F
:103D60000401300E822724EC0BF031C182F40401EF
:103D7000300E822724EC0BF032C182F40401300EA5
:103D8000822724EC0BF033C182F40401300E822729
:103D900024EC0BF004012C0E826F24EC0BF0200EAF
:103DA000F86EF76AF66A04010900F5CF82F424EC94
:103DB0000BF00900F5CF82F424EC0BF00900F5CFED
:103DC00082F424EC0BF00900F5CF82F424EC0BF024
:103DD0000900F5CF82F424EC0BF00900F5CF82F452
:103DE00024EC0BF00900F5CF82F424EC0BF0090071
:103DF000F5CF82F424EC0BF02EEC0BF044EF23F023
:103E00008351630AD8A444EF23F08451610AD8A4F3
:103E100044EF23F085516C0AD8A444EF23F0865177
:103E2000410A42E08651440A1BE08651420AD8B456
:103E300067EF1FF08651350AD8B4CEEF24F08651D3
:103E4000360AD8B423EF25F08651370AD8B48CEF60
:103E500025F08651380AD8B4EAEF25F044EF23F074
:103E60000798079A04017A0E826F24EC0BF0040184
:103E7000780E826F24EC0BF00401640E826F24EC48
:103E80000BF081A84BEF1FF00401550E826F24EC5C
:103E90000BF050EF1FF004014C0E826F24EC0BF07E
:103EA0002EEC0BF044EF23F00788079A04017A0EFA
:103EB000826F24EC0BF00401410E826F24EC0BF0B6
:103EC0000401610E826F24EC0BF041EF1FF00798A4
:103ED000078A04017A0E826F24EC0BF00401420E73
:103EE000826F24EC0BF00401610E826F24EC0BF066
:103EF00041EF1FF00101666785EF1FF0676785EFEF
:103F00001FF0686785EF1FF069679DEF1FF04F672F
:103F100091EF1FF0506791EF1FF0516791EF1FF085
:103F200052679DEF1FF00101000E006F000E016F40
:103F3000000E026F000E036F12000101620E046F8B
:103F4000010E056F000E066F000E076F66C100F1CF
:103F500067C101F168C102F169C103F1F7EC29F011
:103F600003BF21EF20F00101000E046FA80E056FC2
:103F7000550E066F020E076F66C100F167C101F1B1
:103F800068C102F169C103F166C186F167C187F1B9
:103F900068C188F169C189F1F7EC29F003BFDAEF54
:103FA0001FF00101000E866FA80E876F550E886FF7
:103FB000020E896F0E0EF6EC07F0E8CF18F10F0E27
:103FC000F6EC07F0E8CF19F1100EF6EC07F0E8CFA9
:103FD0001AF1110EF6EC07F0E8CF1BF140EC29F0D6
:103FE00086C104F187C105F188C106F189C107F1D5
:103FF000F7EC29F0078204EC29F040EC29F0079255
:1040000004EC29F086C100F187C101F188C102F1F9
:1040100089C103F1079204EC29F0CC0E046FE00E85
:10402000056F870E066F050E076FF7EC29F000C1CC
:1040300018F101C119F102C11AF103C11BF159EFC5
:1040400020F00101800E006F1A0E016F060E026F44
:10405000000E036F4FC104F150C105F151C106F1CB
:1040600052C107F1F7EC29F003AF3AEF20F0F2EC80
:104070002AF012000E0EF6EC07F0E8CF18F10F0E42
:10408000F6EC07F0E8CF19F1100EF6EC07F0E8CFE8
:104090001AF1110EF6EC07F0E8CF1BF14FC100F159
:1040A00050C101F151C102F152C103F1078204EC88
:1040B00029F018C100F119C101F11AC102F11BC1A7
:1040C00003F112000401730E826F24EC0BF0040163
:1040D0002C0E826F24EC0BF0078462C166F163C181
:1040E00067F164C168F165C169F14BC14FF14CC121
:1040F00050F14DC151F14EC152F157C159F158C162
:104100005AF1079488EC20F02EEC0BF044EF23F0EA
:1041100066C100F167C101F168C102F169C103F133
:10412000010195EC2AF078EC28F00401630E826F0F
:1041300024EC0BF004012C0E826F24EC0BF04FC129
:1041400000F150C101F151C102F152C103F101016D
:1041500095EC2AF078EC28F00401660E826F24ECCE
:104160000BF004012C0E826F24EC0BF0F2EC2AF021
:1041700059C100F15AC101F1010195EC2AF078EC26
:1041800028F00401740E826F24EC0BF012001082F0
:104190000401530E826F24EC0BF004012C0E826F8D
:1041A00024EC0BF083C32AF184C32BF185C32CF1DB
:1041B00086C32DF187C32EF188C32FF189C330F157
:1041C0008AC331F18BC332F18CC333F1010140EC6E
:1041D0002BF0B7EC2AF000C166F101C167F102C112
:1041E00068F103C169F18EC32AF18FC32BF190C32B
:1041F0002CF191C32DF192C32EF193C32FF194C3EF
:1042000030F195C331F196C332F197C333F1010117
:1042100040EC2BF0B7EC2AF000C14FF101C150F196
:1042200002C151F103C152F133EC2BF099C32FF1CC
:104230009AC330F19BC331F19CC332F19DC333F17A
:10424000010140EC2BF0B7EC2AF000C159F101C19B
:104250005AF188EC20F004012C0E826F24EC0BF054
:1042600039EF21F08251520A03E10F8239EF21F038
:104270000F928251750A03E1108440EF21F01094EF
:104280008251550A03E1108647EF21F0109607840A
:1042900010B2A4EF21F010A490EF21F0B6C166F1A6
:1042A000B7C167F1B8C168F1B9C169F1BAC16AF1C2
:1042B000BBC16BF1BCC16CF1BDC16DF1BEC16EF192
:1042C000BFC16FF1C0C170F1C1C171F1C2C172F162
:1042D000C3C173F1C4C174F1C5C175F1C6C176F132
:1042E000C7C177F1C8C178F1C9C179F1CAC17AF102
:1042F000CBC17BF1CCC17CF1CDC17DF1CEC17EF1D2
:10430000CFC17FF1D0C180F1D1C181F1D2C182F1A1
:10431000D3C183F1D4C184F1D5C185F198EF21F0E7
:1043200062C166F163C167F164C168F165C169F199
:104330004BC14FF14CC150F14DC151F14EC152F141
:1043400057C159F158C15AF107940FA0C6EF21F097
:1043500001019267B3EF21F09367B3EF21F0946707
:10436000B3EF21F09567B7EF21F0C6EF21F07AECBB
:104370001FF092C104F193C105F194C106F195C1FA
:1043800007F1F7EC29F003BF0AEF23F07AEC1FF0F6
:104390000101000E046F000E056F010E066F000E86
:1043A000076F28EC2AF010A4DDEF21F00401750E50
:1043B000826F24EC0BF0E2EF21F00401720E826FA9
:1043C00024EC0BF004012C0E826F24EC0BF095EC26
:1043D0002AF02967F1EF21F00401200E826FF4EF3B
:1043E00021F004012D0E826F24EC0BF030C182F419
:1043F0000401300E822724EC0BF031C182F4040159
:10440000300E822724EC0BF004012E0E826F24EC78
:104410000BF032C182F40401300E822724EC0BF041
:1044200033C182F40401300E822724EC0BF0040126
:104430006D0E826F24EC0BF004012C0E826F24ECC5
:104440000BF04FC100F150C101F151C102F152C155
:1044500003F1010195EC2AF078EC28F00401480EF4
:10446000826F24EC0BF004017A0E826F24EC0BF0C7
:1044700004012C0E826F24EC0BF066C100F167C1C1
:1044800001F168C102F169C103F1010195EC2AF063
:1044900078EC28F00401630E826F24EC0BF0040129
:1044A0002C0E826F24EC0BF066C100F167C101F1A4
:1044B00068C102F169C103F101010A0E046F000E27
:1044C000056F000E066F000E076F08EC2AF0000E55
:1044D000046F120E056F000E066F000E076F28ECBA
:1044E0002AF095EC2AF02AC182F40401300E8227CA
:1044F00024EC0BF02BC182F40401300E822724EC53
:104500000BF02CC182F40401300E822724EC0BF056
:104510002DC182F40401300E822724EC0BF02EC151
:1045200082F40401300E822724EC0BF02FC182F4B8
:104530000401300E822724EC0BF030C182F4040118
:10454000300E822724EC0BF004012E0E826F24EC37
:104550000BF031C182F40401300E822724EC0BF001
:1045600032C182F40401300E822724EC0BF033C1F7
:1045700082F40401300E822724EC0BF00401730E48
:10458000826F24EC0BF004012C0E826F24EC0BF0F4
:10459000F2EC2AF059C100F15AC101F16EEC24F09D
:1045A0000FB2D6EF22F00FA008EF23F004012C0E7B
:1045B000826F24EC0BF0200EF86EF76AF66A0401A5
:1045C0000900F5CF82F424EC0BF00900F5CF82F45A
:1045D00024EC0BF00900F5CF82F424EC0BF0090079
:1045E000F5CF82F424EC0BF00900F5CF82F424EC33
:1045F0000BF00900F5CF82F424EC0BF00900F5CFA5
:1046000082F424EC0BF00900F5CF82F424EC0BF0DB
:104610002EEC0BF00F9044EF23F00401630E826F39
:1046200024EC0BF004012C0E826F24EC0BF04AEC0E
:1046300023F004012C0E826F24EC0BF0BDEC23F070
:1046400004012C0E826F24EC0BF039EC24F00401F1
:104650002C0E826F24EC0BF00101F80E006FCD0ED2
:10466000016F660E026F030E036F5FEC23F004010F
:104670002C0E826F24EC0BF04FEC24F02EEC0BF0A0
:1046800044EF23F02EEC0BF00301C26B0790109265
:1046900053EF26F0D8900E0EF6EC07F0E8CF00F1BD
:1046A0000F0EF6EC07F0E8CF01F1100EF6EC07F074
:1046B000E8CF02F1110EF6EC07F0E8CF03F10101AB
:1046C000000E046F000E056F010E066F000E076FDF
:1046D00028EC2AF095EC2AF02AC182F40401300E6D
:1046E000822724EC0BF02BC182F40401300E8227C8
:1046F00024EC0BF02CC182F40401300E822724EC50
:104700000BF02DC182F40401300E822724EC0BF053
:104710002EC182F40401300E822724EC0BF02FC14D
:1047200082F40401300E822724EC0BF030C182F4B5
:104730000401300E822724EC0BF031C182F4040115
:10474000300E822724EC0BF004012E0E826F24EC35
:104750000BF032C182F40401300E822724EC0BF0FE
:1047600033C182F40401300E822724EC0BF00401E3
:104770006D0E826F24EC0BF01200120EF6EC07F0B7
:10478000E8CF00F1130EF6EC07F0E8CF01F1140EBC
:10479000F6EC07F0E8CF02F1150EF6EC07F0E8CFE3
:1047A00003F101010A0E046F000E056F000E066F83
:1047B000000E076F08EC2AF0000E046F120E056F52
:1047C000000E066F000E076F28EC2AF095EC2AF019
:1047D0002AC182F40401300E822724EC0BF02BC195
:1047E00082F40401300E822724EC0BF02CC182F4F9
:1047F0000401300E822724EC0BF02DC182F4040159
:10480000300E822724EC0BF02EC182F40401300E0E
:10481000822724EC0BF02FC182F40401300E822792
:1048200024EC0BF030C182F40401300E822724EC1A
:104830000BF004012E0E826F24EC0BF031C182F4D8
:104840000401300E822724EC0BF032C182F4040103
:10485000300E822724EC0BF033C182F40401300EB9
:10486000822724EC0BF00401730E826F24EC0BF012
:1048700012000A0EF6EC07F0E8CF00F10B0EF6EC92
:1048800007F0E8CF01F10C0EF6EC07F0E8CF02F1EB
:104890000D0EF6EC07F0E8CF03F16EEF24F0060EF4
:1048A000F6EC07F0E8CF00F1070EF6EC07F0E8CFE2
:1048B00001F1080EF6EC07F0E8CF02F1090EF6EC74
:1048C00007F0E8CF03F16EEF24F00101F2EC2AF0DB
:1048D000078457C100F158C101F107940101E80EA6
:1048E000046F800E056F000E066F000E076F08EC58
:1048F0002AF0000E046F040E056F000E066F000E06
:10490000076F28EC2AF0880E046F130E056F000E57
:10491000066F000E076FF7EC29F00A0E046F000E09
:10492000056F000E066F000E076F28EC2AF095EC5D
:104930002AF001012967A2EF24F00401200E826F02
:10494000A5EF24F004012D0E826F24EC0BF030C192
:1049500082F40401300E822724EC0BF031C182F482
:104960000401300E822724EC0BF032C182F40401E2
:10497000300E822724EC0BF004012E0E826F24EC03
:104980000BF033C182F40401300E822724EC0BF0CB
:104990000401430E826F24EC0BF0120087C32AF14E
:1049A00088C32BF189C32CF18AC32DF18BC32EF15F
:1049B0008CC32FF18DC330F18EC331F190C332F12E
:1049C00091C333F10101296B40EC2BF0B7EC2AF0D5
:1049D0000101000E046F000E056F010E066F000E40
:1049E000076F08EC2AF00E0E0C6E00C10BF0DFEC26
:1049F00007F00F0E0C6E01C10BF0DFEC07F0100E8C
:104A00000C6E02C10BF0DFEC07F0110E0C6E03C14F
:104A10000BF0DFEC07F004017A0E826F24EC0BF050
:104A200004012C0E826F24EC0BF00401350E826F12
:104A300024EC0BF004012C0E826F24EC0BF04AECFA
:104A400023F050EF1FF087C32AF188C32BF189C3ED
:104A50002CF18AC32DF18BC32EF18CC32FF18DC3A2
:104A600030F18EC331F190C332F191C333F10101C2
:104A7000296B40EC2BF0B7EC2AF0880E046F130E74
:104A8000056F000E066F000E076FFCEC29F0000E9C
:104A9000046F040E056F000E066F000E076F08EC22
:104AA0002AF00101E80E046F800E056F000E066FFC
:104AB000000E076F28EC2AF00A0E0C6E00C10BF0F6
:104AC000DFEC07F00B0E0C6E01C10BF0DFEC07F012
:104AD0000C0E0C6E02C10BF0DFEC07F00D0E0C6E2D
:104AE00003C10BF0DFEC07F004017A0E826F24ECB7
:104AF0000BF004012C0E826F24EC0BF00401360E37
:104B0000826F24EC0BF004012C0E826F24EC0BF06E
:104B100039EC24F050EF1FF087C32AF188C32BF142
:104B200089C32CF18AC32DF18BC32EF18CC32FF1D5
:104B30008DC330F18FC331F190C332F191C333F1A2
:104B4000010140EC2BF0B7EC2AF0000E046F120EBE
:104B5000056F000E066F000E076F08EC2AF00101CA
:104B60000A0E046F000E056F000E066F000E076F31
:104B700028EC2AF0120E0C6E00C10BF0DFEC07F0EF
:104B8000130E0C6E01C10BF0DFEC07F0140E0C6E6F
:104B900002C10BF0DFEC07F0150E0C6E03C10BF039
:104BA000DFEC07F004017A0E826F24EC0BF00401B5
:104BB0002C0E826F24EC0BF00401370E826F24EC74
:104BC0000BF004012C0E826F24EC0BF0BDEC23F0F3
:104BD00050EF1FF087C32AF188C32BF189C32CF152
:104BE0008AC32DF18BC32EF18CC32FF18DC330F10D
:104BF0008EC331F190C332F191C333F10101296BBE
:104C000040EC2BF0B7EC2AF0880E046F130E056F02
:104C1000000E066F000E076FFCEC29F0000E046F0B
:104C2000040E056F000E066F000E076F08EC2AF0E9
:104C30000101E80E046F800E056F000E066F000E76
:104C4000076F28EC2AF0060E0C6E00C10BF0DFECAB
:104C500007F0070E0C6E01C10BF0DFEC07F0080E39
:104C60000C6E02C10BF0DFEC07F0090E0C6E03C1F5
:104C70000BF0DFEC07F004017A0E826F24EC0BF0EE
:104C800004012C0E826F24EC0BF00401380E826FAD
:104C900024EC0BF004012C0E826F24EC0BF04FEC93
:104CA00024F050EF1FF081A811EF27F007A8CAEFFA
:104CB00026F00101800E006F1A0E016F060E026FC2
:104CC000000E036F4BC104F14CC105F14DC106F15B
:104CD0004EC107F1F7EC29F003BF11EF27F072EC9A
:104CE00028F04BC100F14CC101F14DC102F14EC1A0
:104CF00003F1078204EC29F018C104F119C105F190
:104D00001AC106F11BC107F1F80E006FCD0E016F3D
:104D1000660E026F030E036FF7EC29F00E0E0C6E99
:104D200000C10BF0DFEC07F00F0E0C6E01C10BF0B1
:104D3000DFEC07F0100E0C6E02C10BF0DFEC07F099
:104D4000110E0C6E03C10BF0DFEC07F007840101BC
:104D5000F2EC2AF057C100F158C101F107940A0E94
:104D60000C6E00C10BF0DFEC07F00B0E0C6E01C1F6
:104D70000BF0DFEC07F00C0E0C6E02C10BF0DFEC59
:104D800007F00D0E0C6E03C10BF0DFEC07F0079877
:104D900011EF27F007AA11EF27F007840101F2ECC9
:104DA0002AF057C100F158C101F10794060E0C6EAC
:104DB00000C10BF0DFEC07F0070E0C6E01C10BF029
:104DC000DFEC07F0080E0C6E02C10BF0DFEC07F011
:104DD000090E0C6E03C10BF0DFEC07F0078462C113
:104DE00000F163C101F164C102F165C103F10794EF
:104DF000120E0C6E00C10BF0DFEC07F0130E0C6E00
:104E000001C10BF0DFEC07F0140E0C6E02C10BF0C9
:104E1000DFEC07F0150E0C6E03C10BF0DFEC07F0B2
:104E2000079A0401805181197F0B0BE09EA809D0DD
:104E300014EE00F081517F0BE126E750812B0F012A
:104E4000AD6E05012F51010A13E081AA38EF27F05A
:104E500005012F51000A0AE00FB838EF27F00501CD
:104E6000306738EF27F00FB838EF27F018EF35F03C
:104E700081B84DEF27F05BEC2DF005012F51020AB0
:104E800002E04DEF27F05C2F4DEF27F05BC55CF59E
:104E90000501010E306F3C0E316F83EF0AF0060101
:104EA0003251385D3351D8A0010F395D800BD8A441
:104EB0005EEF27F032C638F633C639F61200060127
:104EC0003251365D3351D8A0010F375D800BD8B415
:104ED0006EEF27F032C636F633C637F61200078477
:104EE0001AC632F61BC633F61CC638F61DC639F68E
:104EF0004FEC27F01EC632F61FC633F64FEC27F0F4
:104F000020C632F621C633F64FEC27F01AC632F629
:104F10001BC633F61CC636F61DC637F65FEC27F007
:104F20001EC632F61FC633F65FEC27F020C632F6F7
:104F300021C633F65FEC27F03851365F3951D8A0DF
:104F40003929375FF2EC2AF036C600F137C601F195
:104F5000FEEC2AF000C13AF601C13BF622C632F659
:104F600023C633F624C638F625C639F64FEC27F0AB
:104F700026C632F627C633F64FEC27F028C632F69F
:104F800029C633F64FEC27F022C632F623C633F695
:104F900024C636F625C637F65FEC27F026C632F66D
:104FA00027C633F65FEC27F028C632F629C633F65B
:104FB0005FEC27F03851365F3951D8A03929375F77
:104FC000F2EC2AF036C600F137C601F1FEEC2AF009
:104FD00000C13CF601C13DF62AC632F62BC633F6B7
:104FE0002CC638F62DC639F64FEC27F02EC632F611
:104FF0002FC633F64FEC27F030C632F631C633F603
:105000004FEC27F02AC632F62BC633F62CC636F6FE
:105010002DC637F65FEC27F02EC632F62FC633F6D4
:105020005FEC27F030C632F631C633F65FEC27F07E
:105030003851365F3951D8A03929375FF2EC2AF060
:1050400036C600F137C601F1FEEC2AF000C13EF68B
:1050500001C13FF63AC632F63BC633F63CC636F6D9
:105060003DC637F65FEC27F03EC632F63FC633F654
:105070005FEC27F00794120018C100F119C101F18B
:105080001AC102F11BC103F1000E046F000E056F7F
:10509000010E066F000E076F28EC2AF029A167EFBA
:1050A00028F02051D8B467EF28F018C100F119C1D9
:1050B00001F11AC102F11BC103F1000E046F000ED1
:1050C000056F0A0E066F000E076F28EC2AF012001B
:1050D0000101045100130551011306510213075138
:1050E000031312000101186B196B1A6B1B6B120072
:1050F0002AC182F40401300E822724EC0BF02BC16C
:1051000082F40401300E822724EC0BF02CC182F4CF
:105110000401300E822724EC0BF02DC182F404012F
:10512000300E822724EC0BF02EC182F40401300EE5
:10513000822724EC0BF02FC182F40401300E822769
:1051400024EC0BF030C182F40401300E822724ECF1
:105150000BF031C182F40401300E822724EC0BF0F5
:1051600032C182F40401300E822724EC0BF033C1EB
:1051700082F40401300E822724EC0BF012002FC1C0
:1051800082F40401300E822724EC0BF030C182F44B
:105190000401300E822724EC0BF031C182F40401AB
:1051A000300E822724EC0BF032C182F40401300E61
:1051B000822724EC0BF033C182F40401300E8227E5
:1051C00024EC0BF01200060E116E060E126E060E87
:1051D000136E112EE9EF28F0122EE9EF28F0132EAE
:1051E000E9EF28F08B84020E116E020E126E020E91
:1051F000136E112EF9EF28F0122EF9EF28F0132E6E
:10520000F9EF28F08B9412000101005305E10153DE
:1052100003E1025301E1002BC7EC29F0F2EC2AF084
:105220003951006F3A51016F420E046F4B0E056FFA
:10523000000E066F000E076F08EC2AF000C104F1A3
:1052400001C105F102C106F103C107F118C100F166
:1052500019C101F11AC102F11BC103F107B235EF07
:1052600029F0FCEC29F037EF29F0F7EC29F000C128
:1052700018F101C119F102C11AF103C11BF11200A9
:10528000F2EC2AF059C100F15AC101F1060EF6EC18
:1052900007F0E8CF04F1070EF6EC07F0E8CF05F1D0
:1052A000080EF6EC07F0E8CF06F1090EF6EC07F071
:1052B000E8CF07F1F7EC29F000C124F101C125F195
:1052C00002C126F103C127F1290E046F000E056FFC
:1052D000000E066F000E076F08EC2AF0EE0E046F4A
:1052E000430E056F000E066F000E076FFCEC29F0F1
:1052F00024C104F125C105F126C106F127C107F13A
:1053000008EC2AF000C11CF101C11DF102C11EF11F
:1053100003C11FF1120EF6EC07F0E8CF04F1130EF3
:10532000F6EC07F0E8CF05F1140EF6EC07F0E8CF45
:1053300006F1150EF6EC07F0E8CF07F10D0E006F41
:10534000000E016F000E026F000E036F08EC2AF0D2
:10535000180E046F000E056F000E066F000E076F2B
:1053600028EC2AF01CC104F11DC105F11EC106F193
:105370001FC107F1FCEC29F06A0E046F2A0E056FBD
:10538000000E066F000E076FF7EC29F01200BF0E3B
:10539000FA6E200E3A6F396BD8900037013702371A
:1053A0000337D8B0D8EF29F03A2FCDEF29F03907DD
:1053B0003A070353D8B412000331070B80093F6F3B
:1053C00003390F0B010F396F80EC5FF0406F390527
:1053D00080EC5FF0405D405F396B3F33D8B03927D8
:1053E00039333FA9EDEF29F040513927120001016F
:1053F00017EC2BF0D8B01200010103510719346FDC
:10540000DAEC2AF0D8900751031934AF800F12005C
:105410000101346BFEEC2AF0D8A014EC2BF0D8B0CC
:105420001200E9EC2AF0F2EC2AF01F0E366F2AEC9B
:105430002BF00B35D8B0DAEC2AF0D8A00335D8B071
:105440001200362F17EF2AF034B101EC2BF01200C6
:105450000101346B04510511061107110008D8A091
:10546000FEEC2AF0D8A014EC2BF0D8B01200086B98
:10547000096B0A6B0B6B2AEC2BF01F0E366F2AECB4
:105480002BF007510B5DD8A452EF2AF006510A5DAC
:10549000D8A452EF2AF00551095DD8A452EF2AF0A2
:1054A0000451085DD8A065EF2AF00451085F05514A
:1054B000D8A0053D095F0651D8A0063D0A5F0751F7
:1054C000D8A0073D0B5FD8900081362F3FEF2AF020
:1054D00034B101EC2BF0346BFEEC2AF0D8902EECBA
:1054E0002BF007510B5DD8A482EF2AF006510A5D1C
:1054F000D8A482EF2AF00551095DD8A482EF2AF0E2
:105500000451085DD8A091EF2AF0003F91EF2AF0F6
:10551000013F91EF2AF0023F91EF2AF0032BD8B41C
:10552000120034B101EC2BF012000101346BFEECDF
:105530002AF0D8B0120033EC2BF0200E366F003773
:1055400001370237033711EE33F00A0E376FE736B3
:105550000A0EE75CD8B0E76EE552372FA7EF2AF0C6
:10556000362F9FEF2AF034B12981D8901200010123
:105570000A0E346F200E366F11EE29F03451376F5A
:105580000A0ED890E652D8B0E726E732372FC2EF9E
:105590002AF00333023301330033362FBCEF2AF0F5
:1055A000E750FF0FD8A00335D8B0120029B101ECA5
:1055B0002BF01200045100270551D8B0053D0127FA
:1055C0000651D8B0063D02270751D8B0073D032742
:1055D00012000051086F0151096F02510A6F035107
:1055E0000B6F12000101006B016B026B036B120069
:1055F0000101046B056B066B076B12000335D8A025
:1056000012000351800B001F011F021F031F003FE8
:1056100011EF2BF0013F11EF2BF0023F11EF2BF0B8
:10562000032B342B032512000735D8A01200075195
:10563000800B041F051F061F071F043F27EF2BF0D9
:10564000053F27EF2BF0063F27EF2BF0072B342BDE
:1056500007251200003701370237033708370937AB
:105660000A370B3712000101296B2A6B2B6B2C6B4D
:105670002D6B2E6B2F6B306B316B326B336B1200DB
:1056800001012A510F0B2A6F2B510F0B2B6F2C513D
:105690000F0B2C6F2D510F0B2D6F2E510F0B2E6FEB
:1056A0002F510F0B2F6F30510F0B306F31510F0BEC
:1056B000316F32510F0B326F33510F0B336F1200BA
:1056C000899C000EC76E200EC66E9E96C69EC50EA5
:1056D000C96EFF0E9EB602D0E82EFCD79E96C69EDF
:1056E000000EC96EFF0E9EB602D0E82EFCD7C9CFC1
:1056F00000F69E96C69E000EC96EFF0E9EB602D0A4
:10570000E82EFCD7C9CF01F6898C1200000EC76EB7
:10571000200EC66E899C9E96C69EC80EC96EFF0E50
:105720009EB602D0E82EFCD79E96C69E000EC96E8D
:10573000FF0E9EB602D0E82EFCD7C9CF02F69E9689
:10574000C69E000EC96EFF0E9EB602D0E82EFCD794
:10575000C9CF03F6898C899C9E96C69ECA0EC96ED7
:10576000FF0E9EB602D0E82EFCD79E96C69E000E77
:10577000C96EFF0E9EB602D0E82EFCD7C9CF0AF63E
:105780009E96C69E000EC96EFF0E9EB602D0E82EF3
:10579000FCD7C9CF0BF6898C899C9E96C69ECC0EF1
:1057A000C96EFF0E9EB602D0E82EFCD79E96C69E0E
:1057B000000EC96EFF0E9EB602D0E82EFCD7C9CFF0
:1057C00012F69E96C69E000EC96EFF0E9EB602D0C1
:1057D000E82EFCD7C9CF13F6898C1200000EC76ED5
:1057E000200EC66E899C9E96C69EE80EC96EFF0E60
:1057F0009EB602D0E82EFCD79E96C69E000EC96EBD
:10580000FF0E9EB602D0E82EFCD7C9CF1AF69E96A0
:10581000C69E000EC96EFF0E9EB602D0E82EFCD7C3
:10582000C9CF1BF6898C899C9E96C69EEA0EC96ECE
:10583000FF0E9EB602D0E82EFCD79E96C69E000EA6
:10584000C96EFF0E9EB602D0E82EFCD7C9CF22F655
:105850009E96C69E000EC96EFF0E9EB602D0E82E22
:10586000FCD7C9CF23F6898C899C9E96C69EEC0EE8
:10587000C96EFF0E9EB602D0E82EFCD79E96C69E3D
:10588000000EC96EFF0E9EB602D0E82EFCD7C9CF1F
:105890002AF69E96C69E000EC96EFF0E9EB602D0D8
:1058A000E82EFCD7C9CF2BF6898C1200000EC76EEC
:1058B000200EC66E899C9E96C69E240EC96EFF0E53
:1058C0009EB602D0E82EFCD79E96C69EE40EC96E08
:1058D000FF0E9EB602D0E82EFCD7898C899C9E963E
:1058E000C69E200EC96EFF0E9EB602D0E82EFCD7D3
:1058F0009E96C69E5F0EC96EFF0E9EB602D0E82E23
:10590000FCD7898C899C9E96C69E210EC96EFF0E7F
:105910009EB602D0E82EFCD79E96C69EC00EC96EDB
:10592000FF0E9EB602D0E82EFCD7898C899C9E96ED
:10593000C69E260EC96EFF0E9EB602D0E82EFCD77C
:105940009E96C69E000EC96EFF0E9EB602D0E82E31
:10595000FCD7898C12008984000EC76E220EC66E99
:105960009E96C69E000EC96EFF0E9EB602D0E82E11
:10597000FCD79E96C69E000EC96EFF0E9EB602D044
:10598000E82EFCD7C9CFABF59E96C69E000EC96E19
:10599000FF0E9EB602D0E82EFCD7C9CFACF59E967E
:1059A000C69E000EC96EFF0E9EB602D0E82EFCD732
:1059B000C9CFADF59E96C69E000EC96EFF0E9EB66F
:1059C00002D0E82EFCD7C9CFAEF59E96C69E000E3B
:1059D000C96EFF0E9EB602D0E82EFCD7C9CFAFF538
:1059E0009E96C69E000EC96EFF0E9EB602D0E82E91
:1059F000FCD7C9CFB0F59E96C69E000EC96EFF0EAD
:105A00009EB602D0E82EFCD7C9CFB1F589945EECE2
:105A10002FF012008984000EC76E220EC66E9E966D
:105A2000C69E800EC96EFF0E9EB602D0E82EFCD731
:105A30009E96C69EABC5C9FFFF0E9EB602D0E82E4D
:105A4000FCD79E96C69EACC5C9FFFF0E9EB602D07F
:105A5000E82EFCD79E96C69EADC5C9FFFF0E9EB62A
:105A600002D0E82EFCD79E96C69EAEC5C9FFFF0E9B
:105A70009EB602D0E82EFCD79E96C69EAFC5C9FF43
:105A8000FF0E9EB602D0E82EFCD79E96C69EB0C5ED
:105A9000C9FFFF0E9EB602D0E82EFCD79E96C69E8A
:105AA000B1C5C9FFFF0E9EB602D0E82EFCD789947F
:105AB0005EEC2FF012008984000EC76E220EC66EB7
:105AC0009E96C69E070EC96EFF0E9EB602D0E82EA9
:105AD000FCD79E96C69E000EC96EFF0E9EB602D0E3
:105AE000E82EFCD7C9CFABF59E96C69E000EC96EB8
:105AF000FF0E9EB602D0E82EFCD7C9CFACF59E961D
:105B0000C69E000EC96EFF0E9EB602D0E82EFCD7D0
:105B1000C9CFADF59E96C69E000EC96EFF0E9EB60D
:105B200002D0E82EFCD7C9CFAEF589945EEC2FF0F9
:105B30008984000EC76E220EC66E9E96C69E0F0EFC
:105B4000C96EFF0E9EB602D0E82EFCD79E96C69E6A
:105B5000000EC96EFF0E9EB602D0E82EFCD7C9CF4C
:105B6000B3F589945EEC2FF012008984000EC76EA5
:105B7000220EC66E9E96C69E870EC96EFF0E9EB6FC
:105B800002D0E82EFCD79E96C69EABC5C9FFFF0E7D
:105B90009EB602D0E82EFCD79E96C69EACC5C9FF25
:105BA000FF0E9EB602D0E82EFCD79E96C69EADC5CF
:105BB000C9FFFF0E9EB602D0E82EFCD79E96C69E69
:105BC000AEC5C9FFFF0E9EB602D0E82EFCD7899461
:105BD0005EEC2FF089849E96C69E8F0EC96EFF0ED6
:105BE0009EB602D0E82EFCD79E96C69EB3C5C9FFCE
:105BF000FF0E9EB602D0E82EFCD789945EEC2FF003
:105C000012008984000EC76E220EC66E9E96C69E36
:105C1000870EC96EFF0E9EB602D0E82EFCD79E9668
:105C2000C69E000EC96EFF0E9EB602D0E82EFCD7AF
:105C30009E96C69E800EC96EFF0E9EB602D0E82EBE
:105C4000FCD79E96C69E800EC96EFF0E9EB602D0F1
:105C5000E82EFCD79E96C69E800EC96EFF0E9EB69D
:105C600002D0E82EFCD789945EEC2FF089849E96B2
:105C7000C69E8F0EC96EFF0E9EB602D0E82EFCD7D0
:105C80009E96C69E010EC96EFF0E9EB602D0E82EED
:105C9000FCD789945EEC2FF012008984000EC76E49
:105CA000220EC66E9E96C69E870EC96EFF0E9EB6CB
:105CB00002D0E82EFCD79E96C69E000EC96EFF0E3F
:105CC0009EB602D0E82EFCD79E96C69E000EC96EE8
:105CD000FF0E9EB602D0E82EFCD79E96C69E800E82
:105CE000C96EFF0E9EB602D0E82EFCD79E96C69EC9
:105CF000800EC96EFF0E9EB602D0E82EFCD78994A6
:105D00005EEC2FF089849E96C69E8F0EC96EFF0EA4
:105D10009EB602D0E82EFCD79E96C69E010EC96E96
:105D2000FF0E9EB602D0E82EFCD789945EEC2FF0D1
:105D300012008984000EC76E220EC66E9E96C69E05
:105D40008F0EC96EFF0E9EB602D0E82EFCD75EEC19
:105D50002FF09E96C69E810EC96EFF0E9EB602D093
:105D6000E82EFCD789945EEC2FF08984000EC76E74
:105D7000220EC66E9E96C69E8F0EC96EFF0E9EB6F2
:105D800002D0E82EFCD75EEC2FF09E96C69E010E48
:105D9000C96EFF0E9EB602D0E82EFCD789945EEC49
:105DA0002FF089849E96C69E910EC96EFF0E9EB6F8
:105DB00002D0E82EFCD75EEC2FF09E96C69EA50E74
:105DC000C96EFF0E9EB602D0E82EFCD789945EEC19
:105DD0002FF012008984000EC76E220EC66E9E96AA
:105DE000C69E8F0EC96EFF0E9EB602D0E82EFCD75F
:105DF0005EEC2FF09E96C69E810EC96EFF0E9EB67B
:105E000002D0E82EFCD789945EEC2FF01200898432
:105E1000000EC76E220EC66E9E96C69E8F0EC96E6F
:105E2000FF0E9EB602D0E82EFCD75EEC2FF09E96B9
:105E3000C69E010EC96EFF0E9EB602D0E82EFCD79C
:105E400089945EEC2FF012008984000EC76E220E3A
:105E5000C66E9E96C69E910EC96EFF0E9EB602D06D
:105E6000E82EFCD75EEC2FF09E96C69EA50EC96E5E
:105E7000FF0E9EB602D0E82EFCD789945EEC2FF080
:105E800012008984000EC76E220EC66E9E96C69EB4
:105E9000910EC96EFF0E9EB602D0E82EFCD75EECC6
:105EA0002FF09E96C69E000EC96EFF0E9EB602D0C3
:105EB000E82EFCD789945EEC2FF01200050EE82E38
:105EC000FED712000501256B266B276B286B899A7C
:105ED000400EC76E200EC66E9E96C69E030EC96EFD
:105EE000FF0E9EB602D0E82EFCD79E96C69E27C512
:105EF000C9FFFF0E9EB602D0E82EFCD79E96C69E26
:105F000026C5C9FFFF0E9EB602D0E82EFCD79E968E
:105F1000C69E25C5C9FFFF0E9EB602D0E82EFCD74F
:105F20009E96C69EC952FF0E9EB602D0E82EFCD7A2
:105F3000898A0F01C950FF0A01E1120005012E51A3
:105F4000130A05E005012E51170A0CE012000501A5
:105F5000E00E256FFF0E266F0F0E276F000E286FC5
:105F6000BBEF2FF00501E00E256FFF0E266FFF0E31
:105F7000276F000E286F899A400EC76E200EC66EDE
:105F80009E96C69E030EC96EFF0E9EB602D0E82EE8
:105F9000FCD79E96C69E27C5C9FFFF0E9EB602D0AF
:105FA000E82EFCD79E96C69E26C5C9FFFF0E9EB65C
:105FB00002D0E82EFCD79E96C69E25C5C9FFFF0ECF
:105FC0009EB602D0E82EFCD79E96C69EC952FF0E02
:105FD0009EB602D0E82EFCD7898A0F01C950FF0A6D
:105FE0001DE005012E51130A05E005012E51170A87
:105FF0000BE012000501000E256F000E266F100E3B
:10600000276F000E286F12000501000E256F000E8D
:10601000266F000E276F010E286F12000501256BF9
:10602000266B276B286B05012E51130A05E005012D
:106030002E51170A0CE012000501000E216F000E10
:10604000226F080E236F000E246F30EF30F0050131
:10605000000E216F000E226F800E236F000E246F42
:1060600021C500F122C501F123C502F124C503F1C8
:1060700025C504F126C505F127C506F128C507F198
:1060800068EC28F000C125F501C126F502C127F50D
:1060900003C128F5899A400EC76E200EC66E9E96E3
:1060A000C69E030EC96EFF0E9EB602D0E82EFCD728
:1060B0009E96C69E27C5C9FFFF0E9EB602D0E82E4B
:1060C000FCD79E96C69E26C5C9FFFF0E9EB602D07F
:1060D000E82EFCD79E96C69E25C5C9FFFF0E9EB62C
:1060E00002D0E82EFCD79E96C69EC952FF0E9EB6E1
:1060F00002D0E82EFCD7898AC950FF0A08E104C102
:1061000025F505C126F506C127F507C128F5D89064
:10611000050124332333223321332151E00B216F36
:1061200021679AEF30F022679AEF30F023679AEFF9
:1061300030F0246730EF30F00501200E2527E86AA3
:106140002623E86A2723E86A28231200E86A050163
:106150002E51130A06E005012E51170A0BE0020E1C
:10616000120005012851000A03E12751F00B07E056
:10617000010E120005012851000A01E0010E120073
:1061800029C500F12AC501F12BC502F12CC503F187
:1061900025C504F126C505F127C506F128C507F177
:1061A000F7EC29F003BF1200A6EC30F05FE1899A0A
:1061B000400EC76E200EC66E9E96C69E060EC96E17
:1061C000FF0E9EB602D0E82EFCD7898A899A9E9649
:1061D000C69E020EC96EFF0E9EB602D0E82EFCD7F8
:1061E0009E96C69E27C5C9FFFF0E9EB602D0E82E1A
:1061F000FCD79E96C69E26C5C9FFFF0E9EB602D04E
:10620000E82EFCD79E96C69E25C5C9FFFF0E9EB6FA
:1062100002D0E82EFCD79E96C69E000EC96EFF0ED9
:106220009EB602D0E82EFCD7898A899A9E96C69E91
:10623000050EC96EFF0E9EB602D0E82EFCD79E96C4
:10624000C69EC952FF0E9EB602D0E82EFCD7C9B03A
:106250001FEF31F0898A0501200E2527E86A2623E1
:10626000E86A2723E86A2823C0EF30F01200899AF1
:10627000400EC76E200EC66E9E96C69E060EC96E56
:10628000FF0E9EB602D0E82EFCD7898A899A9E9688
:10629000C69EC70EC96EFF0E9EB602D0E82EFCD772
:1062A000898A0501256B266B276B286B1200899A5A
:1062B000400EC76E200EC66E9E96C69E050EC96E17
:1062C000FF0E9EB602D0E82EFCD79E96C69EC952FF
:1062D000FF0E9EB602D0E82EFCD7C9CF33F5898ACF
:1062E0001200899A400EC76E200EC66E9E96C69EFC
:1062F000B90EC96EFF0E9EB602D0E82EFCD7898A71
:106300001200899A400EC76E200EC66E9E96C69EDB
:10631000AB0EC96EFF0E9EB602D0E82EFCD7898A5E
:10632000FF0EE82EFED71200A6EC30F0D8A4120023
:10633000899A400EC76E200EC66E9E96C69E030EAC
:10634000C96EFF0E9EB602D0E82EFCD79E96C69E62
:1063500027C5C9FFFF0E9EB602D0E82EFCD79E9639
:10636000C69E26C5C9FFFF0E9EB602D0E82EFCD7FA
:106370009E96C69E25C5C9FFFF0E9EB602D0E82E8A
:10638000FCD79E96C69EC952FF0E9EB602D0E82E3E
:10639000FCD7898A0F01C950FF0AD8A48BEF34F0CB
:1063A0000501FE0E336FABEC2CF0ABC534F5ACC57C
:1063B00035F5ADC536F5AEC537F5AFC538F5B0C561
:1063C00039F5B1C53AF50784B6C166F1B7C167F1D1
:1063D000B8C168F1B9C169F14BC14FF14CC150F17D
:1063E0004DC151F14EC152F157C159F158C15AF145
:1063F0007AEC1FF000C13BF501C13CF502C13DF54F
:1064000003C13EF505015D670DEF32F05E670DEFEC
:1064100032F05F670DEF32F0606711EF32F01EEF80
:1064200032F05DC504F15EC505F15FC506F160C5DA
:1064300007F1F7EC29F003BF8BEF34F059C13FF5BA
:106440005AC140F5B5C541F5B6C542F56FEC27F028
:1064500036C645F537C646F50601406737EF32F0D8
:10646000416737EF32F0426737EF32F043673BEF77
:1064700032F04CEF32F0F2EC2AF0F8EC2AF036C6AB
:1064800000F137C601F140C604F141C605F1F7EC51
:1064900029F003AF8BEF34F00101036B026B1AC6D6
:1064A00000F11BC601F101AF5AEF32F0FF0E026F8F
:1064B000FF0E036F0101076B066B1CC604F11DC6BE
:1064C00005F105AF68EF32F0FF0E066FFF0E076FA4
:1064D000FCEC29F00101076B066B1EC604F11FC618
:1064E00005F105AF78EF32F0FF0E066FFF0E076F74
:1064F000FCEC29F00101076B066B20C604F121C6F4
:1065000005F105AF88EF32F0FF0E066FFF0E076F43
:10651000FCEC29F0D890010103330233013300333E
:10652000D8900101033302330133003300C147F532
:1065300001C148F50101036B026B22C600F123C6BD
:1065400001F101AFA8EF32F0FF0E026FFF0E036FF3
:106550000101076B066B24C604F125C605F105AFE2
:10656000B6EF32F0FF0E066FFF0E076FFCEC29F05E
:106570000101076B066B26C604F127C605F105AFBE
:10658000C6EF32F0FF0E066FFF0E076FFCEC29F02E
:106590000101076B066B28C604F129C605F105AF9A
:1065A000D6EF32F0FF0E066FFF0E076FFCEC29F0FE
:1065B000D89001010333023301330033D890010135
:1065C000033302330133003300C149F501C14AF5F9
:1065D0000101036B026B2AC600F12BC601F101AF6A
:1065E000F6EF32F0FF0E026FFF0E036F0101076B33
:1065F000066B2CC604F12DC605F105AF04EF33F090
:10660000FF0E066FFF0E076FFCEC29F00101076B10
:10661000066B2EC604F12FC605F105AF14EF33F05B
:10662000FF0E066FFF0E076FFCEC29F00101076BF0
:10663000066B30C604F131C605F105AF24EF33F027
:10664000FF0E066FFF0E076FFCEC29F0D8900101DA
:106650000333023301330033D89001010333023393
:106660000133003300C14BF501C14CF50101036B4F
:10667000026B02C600F103C601F101AF44EF33F033
:10668000FF0E026FFF0E036F0101076B066B04C65E
:1066900004F105C605F105AF52EF33F0FF0E066FAA
:1066A000FF0E076FFCEC29F00101076B066B06C6B5
:1066B00004F107C605F105AF62EF33F0FF0E066F78
:1066C000FF0E076FFCEC29F00101076B066B08C693
:1066D00004F109C605F105AF72EF33F0FF0E066F46
:1066E000FF0E076FFCEC29F0D89001010333023351
:1066F00001330033D89001010333023301330033F7
:1067000000C14DF501C14EF50101036B026B0AC6D4
:1067100000F10BC601F101AF92EF33F0FF0E026FF3
:10672000FF0E036F0101076B066B0CC604F10DC66B
:1067300005F105AFA0EF33F0FF0E066FFF0E076FF8
:10674000FCEC29F00101076B066B0EC604F10FC6C5
:1067500005F105AFB0EF33F0FF0E066FFF0E076FC8
:10676000FCEC29F00101076B066B10C604F111C6A1
:1067700005F105AFC0EF33F0FF0E066FFF0E076F98
:10678000FCEC29F0D89001010333023301330033CC
:10679000D8900101033302330133003300C14FF5B8
:1067A00001C150F50101036B026B12C600F113C663
:1067B00001F101AFE0EF33F0FF0E026FFF0E036F48
:1067C0000101076B066B14C604F115C605F105AF90
:1067D000EEEF33F0FF0E066FFF0E076FFCEC29F0B3
:1067E0000101076B066B16C604F117C605F105AF6C
:1067F000FEEF33F0FF0E066FFF0E076FFCEC29F083
:106800000101076B066B18C604F119C605F105AF47
:106810000EEF34F0FF0E066FFF0E076FFCEC29F051
:10682000D89001010333023301330033D8900101C2
:10683000033302330133003300C151F501C152F576
:1068400007940501210E326F899A400EC76E200E03
:10685000C66E9E96C69E060EC96EFF0E9EB602D0EE
:10686000E82EFCD7898A899A9E96C69E020EC96E2A
:10687000FF0E9EB602D0E82EFCD79E96C69E27C578
:10688000C9FFFF0E9EB602D0E82EFCD79E96C69E8C
:1068900026C5C9FFFF0E9EB602D0E82EFCD79E96F5
:1068A000C69E25C5C9FFFF0E9EB602D0E82EFCD7B6
:1068B00025EE33F0322F02D069EF34F09E96C69E5B
:1068C000DECFC9FFFF0E9EB602D0E82EFCD75AEFEE
:1068D00034F0898A899A9E96C69E050EC96EFF0E6F
:1068E0009EB602D0E82EFCD79E96C69EC952FF0ED9
:1068F0009EB602D0E82EFCD7C9B074EF34F0898A76
:106900000501200E2527E86A2623E86A2723E86A7E
:106910002823E3EC28F0120021C500F122C501F183
:1069200023C502F124C503F1899A400EC76E200EDB
:10693000C66E9E96C69E0B0EC96EFF0E9EB602D008
:10694000E82EFCD79E96C69E02C1C9FFFF0E9EB6DA
:1069500002D0E82EFCD79E96C69E01C1C9FFFF0E4D
:106960009EB602D0E82EFCD79E96C69E00C1C9FFF7
:10697000FF0E9EB602D0E82EFCD79E96C69EC95248
:10698000FF0E9EB602D0E82EFCD725EE33F00501AF
:10699000200E326F9E96C69EC952FF0E9EB602D042
:1069A000E82EFCD7C9CFDEFF322FCAEF34F0898A38
:1069B0001200899A400EC76E200EC66E9E96C69E25
:1069C000900EC96EFF0E9EB602D0E82EFCD79E96A2
:1069D000C69E000EC96EFF0E9EB602D0E82EFCD7F2
:1069E0009E96C69E000EC96EFF0E9EB602D0E82E81
:1069F000FCD79E96C69E000EC96EFF0E9EB602D0B4
:106A0000E82EFCD79E96C69EC952FF0E9EB602D0B7
:106A1000E82EFCD7C9CF2DF59E96C69EC952FF0E13
:106A20009EB602D0E82EFCD7C9CF2EF5898A120077
:106A3000E3EC28F0B5C5E8FFD70802E3E3EC28F063
:106A4000B5C5E8FFC80802E3E3EC28F0B5C5E8FFE8
:106A5000B90802E3E3EC28F0B5C5E8FFAA0802E3B1
:106A6000E3EC28F0B5C5E8FF9B0802E3E3EC28F06F
:106A70005BEC2DF071EC31F0F29CF29E8B94C69A97
:106A8000C290898C9482948C720ED36ED3A4FED75C
:106A900089968A909390FF0EE8CF00F0E82EFED7FB
:106AA000002EFCD78150F294F29A9E909D909E9277
:106AB0009D92F298F292F290F286F28E0300FF001D
:10BF0000E844F926000C160C2B0C3F0C520C640C68
:10BF1000760C860C960CA50CB30CC10CCF0CDC0C6B
:06BF2000E80CF40C000C1B
:00000001FF
